:100000000C94FD010C941A020C94050C0C941A0229
:100010000C941A020C941A020C941A020C94C60C3A
:100020000C941A020C941A020C941A020C941A02E0
:100030000C941A020C9496080C941A020C941A024E
:100040000C941A020C941A020C941A020C941A02C0
:100050000C941A020C941A020C94A3050C941A0224
:100060000C941A023F065B4F666D7D077F6F777CAD
:10007000395E7971004053332944494E2E000030D7
:10008000280000100800024002C593C08094199413
:1000900098918815981599848095999598000000F5
:1000A000000000000002020000538E9589A4B805EC
:1000B00011A4B01519150905999189202080915135
:1000C000050111C3818385859195098595950D0657
:1000D000142420819141038187420642204412006A
:1000E000000000000000000000040080000080000C
:1000F0001000010100020020004000000800040080
:100100002000021000000000000000E351D1635203
:1001100062E2CDC34FCFD2ADEDF2A8A3B260E061F1
:10012000E19283888DC80444D050E884C4434F4E84
:1001300054494B4900364C4F5750414E0050494EA0
:10014000470050494E47494E470054454D50004DD9
:100150004F4445200044454720460044454720433E
:100160000053454E44004F4E4345004155544F0007
:10017000444542554700444247204F4E00444247C1
:10018000204F46460053454E540053454E44494E79
:1001900047002D01000200000000000035010002B0
:1001A0000000000000003D0100030B040000980B5C
:1001B000420102020202000000004A010005020B97
:1001C000000000004F01040608080000000055016F
:1001D000050507070100440B5B0105050606000045
:1001E000440B610104090505000000006601080ECA
:1001F0000A0A0000020B6B01080F09090100020B3B
:100200007001000C04020000000076010B0B0D0DC4
:100210000100540B7D010B0B0C0C0000540B8501ED
:10022000090E0E0E000000008A010A0F0F0F0000D9
:10023000000050494E4753204641494C4544005721
:10024000414B452D2D2D009B0395038F0388038281
:10025000037B0373036C0364035C0353034B03428C
:100260000339032F0326031C0312030703FD02F2C5
:1002700002E702DC02D002C502B902AD02A102957A
:100280000289027C027002630257024A023E023275
:1002900002250219020C020002F401E801DC01D07F
:1002A00001C401B801AD01A20196018C0181017662
:1002B000016C01620158014E0144013B01320129E8
:1002C00001200117010F010701FF00F700F000E90D
:1002D00000E100DB00D400CD00C700C100BB00AAD4
:1002E00003A703A403A1039E039B03980394039114
:1002F000038D038A03860382037E037B03770372E5
:10030000036E036A03660361035D03580353034FDF
:10031000034A03450340033B03360330032B032604
:100320000320031B0315030F030A030403FE02F853
:1003300002F202EC02E602DF02D902D302CC02C6CC
:1003400002BF02B902B202AC02A5029E029702915C
:10035000028A0283027C0275026E02680261025AFE
:100360000253024C0245023E0237023002290222A9
:10037000021B0215020E0207020002F901F201EC53
:1003800001E501DE01D801D101CB01C401BE01B7F5
:1003900001B101AA01A4019E01980192018C01867C
:1003A0000180017A0174016E01680163015D0158E9
:1003B0000152014D01470142013D01380133012E37
:1003C00001290124011F011A01150111010C010865
:1003D000010301FF00FB00F600F200EE00EA00E678
:1003E00000E200DE00DB00D700D300CF00CC00C865
:1003F00000C500C200BE00BB000011241FBECFEF2D
:10040000D8E0DEBFCDBF11E0A0E0B1E0E4E5FAE165
:1004100002C005900D92A631B107D9F711E0A6E10F
:10042000B1E001C01D92AD39B107E1F70E940507A7
:100430000C94280D0C940000E4E6F0E090819E7F7F
:100440009083206820937A00482B40937C0060932F
:100450007B0081E0809316011092170180E090E00C
:100460000895EAE7F0E080818F778083E4E6F0E0AA
:100470008081816080831092160110921701089587
:1004800080911601882319F42FEF3FEF0AC081E015
:100490008093170180917A00806480937A0020E035
:1004A00030E0C9010895982F80911701882399F0B1
:1004B00080917A0086FD0FC01092170180917C0018
:1004C0009295990F907E892B80937C0020917800E3
:1004D0003091790002C02FEF3FEFC90108950E94CB
:1004E000400280E00E9453022FEF8F3F9207C9F332
:1004F000629902C080E10895803A910514F481E088
:10050000089521E08038920714F488E0089522E0ED
:100510008038920714F484E008958058934014F0D2
:1005200080E0089582E008950E946F029091350165
:10053000882329F4903249F41092350108959032BD
:1005400011F480E008958093350108950E9494028B
:10055000811181E008950E94A6028823E1F3809131
:10056000350190E29093350108950E94310208957B
:10057000EEE7F0E08081826080836A98729A8198C9
:10058000899827E040E460E081E00E941C02089521
:100590008091E40084FFFCCF81E98093E4008091A6
:1005A000E40084FFFCCF1092E4008091640080613D
:1005B000809364000895482F6AE00E94F50C282F6C
:1005C00030E084E0220F331F8A95E1F7842F0E94E8
:1005D000F50C892F822B089560E070E021C0FA01AC
:1005E0008491E82FF0E0EF71F070E451FF4F20812B
:1005F00082958695877090E0032E02C0880F991F20
:100600000A94E2F78095822380834F5F5F4FF0E08A
:100610004D375F0721F76E5F7F4F6830710521F01E
:10062000362F46E750E0DBCF80E090E00895382F8A
:10063000E82FEF71E43180F4F0E0E451FF4F2081C6
:1006400032953695377081E090E002C0880F991F8F
:100650003A95E2F7282B20830895382FE82FEF7181
:10066000E43188F4F0E0E451FF4F20813295369573
:10067000377081E090E002C0880F991F3A95E2F749
:1006800080958223808308950F931F93CF93DF93E8
:100690009C01CB01820F931F839724F062E270E0EC
:1006A000621B730BD901A55FBE4FA901620F731FB7
:1006B000C1E0D0E018C0FD018491E82FEF71E43172
:1006C00078F4F0E0E451FF4F2081829586958770A1
:1006D0008E0102C0000F111F8A95E2F7202B2083A4
:1006E0004F5F5F4F1196461757072CF3DF91CF915D
:1006F0001F910F9108950F931F93CF93DF939C0148
:10070000CB01820F931F839724F062E270E0621B9B
:10071000730BD901A55FBE4FA901C1E0D0E01AC09B
:10072000FD018491E82FEF71E43188F4F0E0E451A9
:10073000FF4F20818295869587708E0102C0000F41
:10074000111F8A95E2F7C8018095822380834F5F4D
:100750005F4F1196461757071CF3DF91CF911F91FA
:100760000F910895809164008F7E809364008FEFD5
:100770008093E50087E08093E6008EE68093E700B3
:1007800088EC8093E40062E270E080E090E00E94F8
:100790007B0380E290E024E0959587952A95E1F728
:1007A000009711F481E090E090933401809333013D
:1007B000909332018093310180E090E00895CF93CF
:1007C000DF93660F771FA6E7B0E040E050E0C82F48
:1007D000D0E0CE01042E02C0959587950A94E2F7E9
:1007E00080FF16C0FD018491E82FF0E0EF71F070FA
:1007F000E451FF4F208182958695877090E0062E08
:1008000002C0880F991F0A94E2F7282B208316C094
:10081000FD018491E82FF0E0EF71F070E451FF4F9B
:10082000208182958695877090E0062E02C0880F01
:10083000991F0A94E2F78095822380834F5F5F4F70
:1008400011964730510509F0C4CFDF91CF9108953B
:10085000AF92BF92CF92DF92EF92FF920F931F93CE
:10086000CF93DF937C01C62ED42EC0E0D0E000E011
:1008700010E04FE0A42EB12CF501002E02C0EE0FC7
:10088000FF1F0A94E2F7EE21FF21002E02C0F69529
:10089000E7950A94E2F7EC59FF4FE491BE018E2FE1
:1008A0000E94DF032196C430D105C1F10C5F1F4FB8
:1008B000C701002E02C0969587950A94E2F7892B0E
:1008C000D9F6BE01CC2089F02196DD2019F0E5E7AC
:1008D000F0E002C0E4E6F0E084910E94DF03DD2056
:1008E000C9F48091F400806803C08091F4008F7790
:1008F0008093F4000FC0DD2019F0E4E7F0E002C0BF
:10090000E4E6F0E08E010F5F1F4F8491BE010E946C
:10091000DF03E801C430D10574F30BC0CC2021F013
:100920008091F400806803C08091F4008F778093F9
:10093000F40080E090E0DF91CF911F910F91FF9044
:10094000EF90DF90CF90BF90AF900895462F28EDA5
:10095000813F920714F481EF98EDFC0187E2E031CA
:10096000F80714F0EFE0F7E2DF01F7FF04C0AA2771
:10097000BB27AE1BBF0B8A2F6AE00E94F50C282F05
:1009800030E054E0220F331F5A95E1F76F2F661FB6
:100990006627661F96EF899F802D11248A0F822B70
:1009A00090E00E9428040895462F60E00E942804E9
:1009B00008950F931F93CF93DF93982F9B01683077
:1009C00071050CF05EC08A52813520F0903209F03A
:1009D00058C00BC0913608F09F7D903231F0892FBE
:1009E0008A52863308F04DC001C080E0E82FF0E065
:1009F000EE0FFF1FE358FF4F85919591A591B4919C
:100A0000EC01822F81508695A82FB0E0A451BF4FF2
:100A100068E070E440E050E0890101701070FD0171
:100A2000E40FF51FCE018F70382F962F9F7024E0B2
:100A3000D695C7952A95E1F784E0769567958A95CE
:100A4000E1F70115110519F0292F206F06C0329525
:100A5000307F292F2295207F2F6090818081832BEA
:100A60009223892B8083808190812823232B292323
:100A700020834B5F5F4F4431510589F620E030E021
:100A800002C02FEF3FEFC901DF91CF911F910F916E
:100A90000895EF92FF920F931F93CF93DF937C0102
:100AA0008B01C1E0D0E005C0BE0180E20E94D90404
:100AB0002196C017D107C4F3E8010EC0F701808169
:100AC000882319F4BE0180E204C00894E11CF11CE3
:100AD000BE010E94D9042196C830D1057CF380E084
:100AE00090E0DF91CF911F910F91FF90EF900895CB
:100AF0000F931F9300911A0110911B01F801E45EFE
:100B0000FE4F80830F5F1F4F10931B0100931A014C
:100B1000F801E45EFE4F1082809118019091190156
:100B200061E070E0845E9E4F0E94490510923001A2
:100B3000083011051CF081E08093300180E090E0E6
:100B40001F910F9108951F920F920FB60F921124CB
:100B50002F933F934F935F936F937F938F939F93C5
:100B6000AF93BF93EF93FF9380913001882309F4F3
:100B700042C08091310190913201019790933201EE
:100B800080933101892BB9F5209118013091190119
:100B9000F901E45EFE4F8081882339F41092190137
:100BA0001092180187E090E007C0809100019091B9
:100BB0000101009731F001979093010180930001AA
:100BC00006C02F5F3F4F30931901209318016091A9
:100BD0000001709101018091180190911901845ECA
:100BE0009E4F0E944905809133019091340190936A
:100BF000320180933101FF91EF91BF91AF919F91AD
:100C00008F917F916F915F914F913F912F910F90B5
:100C10000FBE0F901F901895279A2F980895279828
:100C20002F9A0895E4E6F0E0E80FF11DE49170E0FA
:100C30008E2F0E94DF0308950F931F938C01BC0138
:100C40008CE191E00E94D50CC8010E94DC0C8C0163
:100C500090931B0180931A011092190110921801B0
:100C600061E070E08CE191E00E9449051092300152
:100C7000083011051CF081E08093300180E090E0A5
:100C80001F910F910895CF92DF92EF92FF920F93F1
:100C90001F93D82EC92E5CE1E52E51E0F52E482F8A
:100CA000592FC7010E94E50C0D2D1C2D10931B011F
:100CB00000931A01109219011092180161E070E07E
:100CC000C7010E94490510923001083011051CF03F
:100CD00081E08093300180E090E01F910F91FF90C0
:100CE000EF90DF90CF9008950F931F93182F092F47
:100CF000682F792F8CE191E00E94EE0CE12FF02F0C
:100D0000DF010D900020E9F78D01015010400E1B0E
:100D10001F0B10931B0100931A01109219011092DE
:100D2000180161E070E08CE191E00E9449051092A9
:100D30003001083011051CF081E08093300180E023
:100D400090E01F910F9108959AE0899FF00111247E
:100D5000EE56FE4FA7E3B1E084918D93319681E08A
:100D6000A134B807C9F708958091370190913801EF
:100D700021E08D329207A1F42CE931E0A7E3B1E044
:100D8000F90184918D932F5F3F4FF1E0A134BF07AC
:100D9000B9F780913701909138010E941C0608959F
:100DA0008553914099F422E931E0A7E3B1E0F901DC
:100DB00084918D932F5F3F4FF1E0A134BF07B9F7C6
:100DC00080913701909138010E941C06089580910E
:100DD0003701909138018A54914011F40E940F0B11
:100DE00080913701909138018B56914011F40E9407
:100DF000C20A80913701909138018D53914021F4BE
:100E00000E94BF0A0E94EC0208951F930E94B20341
:100E10000E94B8020E946E080E947D0B0E944D0C39
:100E20000E94AE0C789483EE0E9417038DEE0E9410
:100E3000170322E931E0A7E3B1E0F90184918D9332
:100E40002F5F3F4FF1E0A134BF07B9F78091370121
:100E5000909138010E941C060E94B80C1AE0789408
:100E600080919C018823C9F110929C010E94B406D4
:100E700080919601882311F00E941D0B80919701AB
:100E8000882311F00E94D60A80919501882329F1C8
:100E900080914101843059F480919901882339F47B
:100EA00010924101109242010E94BF0A16C0809127
:100EB0009901882371F010929901809142018F5F0E
:100EC00080934201843049F482E392E00E941C0640
:100ED00004C00E94C50A809341010E94A602882393
:100EE00009F48CC00E94AB02843089F1853030F463
:100EF000813059F0823009F07FC018C0883009F481
:100F000037C0803109F078C04AC080913B01819F91
:100F1000F0011124EE56FE4FA7E3B1E084918D93CA
:100F2000319681E0A134B807C9F760C080913C01D7
:100F3000819FF0011124EE56FE4FA7E3B1E08491AA
:100F40008D93319681E0A134B807C9F74FC08091E5
:100F50003901819FF0011124EE56FE4FA7E3B1E065
:100F600084918D93319681E0A134B807C9F73EC0D2
:100F700080913F0190914001892B89F480913A0141
:100F8000819FF0011124EE56FE4FA7E3B1E084915A
:100F90008D93319681E0A134B807C9F727C0E0915D
:100FA0003F01F0914001309739F180913D019091DE
:100FB0003E01099580913D0190913E01892B31F0D0
:100FC00080913701909138010E941C0680913A016E
:100FD000819FF0011124EE56FE4FA7E3B1E084910A
:100FE0008D93319681E0A134B807C9F7809137011C
:100FF000909138010E941C060E94E70680E00E9442
:1010000016092DCFFC011182818180830895DC01B6
:101010009C919F5F903508F090E011968C9111970C
:10102000981731F08C91FD01E80FF11D62839C93BC
:101030000895DC0111968C911197FD01E80FF11DC7
:1010400092818F5F803508F080E011968C93892F14
:1010500008951092430180914301809344010895C3
:10106000FC019081818120E0981321E0822F089576
:101070008A3010F0895C0895805D0895FB0190E34B
:1010800090838F708A3010F0895C01C0805D81830D
:10109000089520E43BE44CE450E00BC021153105F9
:1010A0004105510511F49FEF17C0215030404040D9
:1010B00050409091430180914401981779F38091B9
:1010C0004401E82FF0E0ED5BFE4F92818F5F8035A9
:1010D00008F080E080934401892F0895E4E6F0E071
:1010E00080818D7F808310924301809143018093A2
:1010F00044018CE090E09093C5008093C40086E0AA
:101100008093C20088E98093C10008951092C100C5
:10111000E4E6F0E08081826080830895982F8091DA
:10112000C00085FFFCCF9093C60008951F920F92D8
:101130000FB60F9211242F938F939F93EF93FF93EA
:101140002091C600909143019F5F903508F090E098
:1011500080914401981741F0E0914301F0E0ED5B8C
:10116000FE4F228390934301FF91EF919F918F91C6
:101170002F910F900FBE0F901F901895982F809170
:10118000C00085FFFCCF81E08093C6008091C00045
:1011900085FFFCCF6093C6008091C00085FFFCCF27
:1011A0009093C600FA0190E009C020818091C000B0
:1011B00085FFFCCF2093C6009F5F31969617A9F755
:1011C0008091C00085FFFCCF84E08093C600089525
:1011D000DF93CF93CDB7DEB764970FB6F894DEBF39
:1011E0000FBECDBF982FDE011196E2E0F1E088E05E
:1011F00001900D928150E1F7FE0139968CE0DF01FC
:101200001D928A95E9F7BE016C5F7F4F892F0E947E
:10121000790ACE0101960E94740664960FB6F8947E
:10122000DEBF0FBECDBFCF91DF910895DF93CF9387
:10123000CDB7DEB72D970FB6F894DEBF0FBECDBF8A
:10124000882399F49091430180914401981769F49F
:1012500047C1211531054105510511F49FEF1CC00F
:10126000215030404040504004C020E43BE44CE476
:1012700050E09091430180914401981751F380917F
:101280004401E82FF0E0ED5BFE4F92818F5F8035E7
:1012900008F080E08093440199838981813011F0C6
:1012A00081E0EDC00E940C0620E43BE44CE450E0F9
:1012B0000BC0211531054105510511F49FEF17C0F1
:1012C0002150304040405040909143018091440172
:1012D000981779F380914401E82FF0E0ED5BFE4F21
:1012E00092818F5F803508F080E08093440199837C
:1012F00089818F3F11F482E0C2C0898187FF2CC0B1
:1013000020E43BE44CE450E00BC0211531054105DD
:10131000510511F49FEF17C021503040404050401C
:101320009091430180914401981779F38091440191
:10133000E82FF0E0ED5BFE4F92818F5F803508F083
:1013400080E08093440199838981843009F4C6C088
:1013500083E00E94E808C2C089818A838A818B3039
:1013600008F0BEC020E43BE44CE450E00BC0211583
:1013700031054105510511F49FEF17C02150304050
:10138000404050409091430180914401981779F377
:1013900080914401E82FF0E0ED5BFE4F92818F5F7A
:1013A000803508F080E080934401998389818F3FE4
:1013B00011F485E064C089818B8360E070E0DE0118
:1013C00014962BC0211531054105510511F49FEFED
:1013D00017C02150304040405040909143018091CF
:1013E0004401981779F380914401E82FF0E0ED5B18
:1013F000FE4F92818F5F803508F080E0809344013A
:10140000998389818F3F11F4862F39C08981FD012D
:10141000E60FF71F80836F5F7F4F8A8190E0681728
:10142000790728F020E43BE44CE450E010C020E4CD
:101430003BE44CE450E0D1CF211531054105510585
:1014400011F49FEF17C02150304040405040909120
:10145000430180914401981779F380914401E82F6A
:10146000F0E0ED5BFE4F92818F5F803508F080E009
:101470008093440199838981843021F087E00E9420
:10148000E8082EC08B81813CD1F0823C09F1803C80
:1014900029F58C8180939B01813011F463E00BC0AE
:1014A000823011F462E007C0833011F461E003C0C0
:1014B000843019F460E00E9412061092990181E5CF
:1014C0000E9417030E94250C81E50E942D0306C08F
:1014D000CE0104960E9474060E94250C0E940F06FD
:1014E0002D960FB6F894DEBF0FBECDBFCF91DF9122
:1014F0000895282FFB016AE00E94F50C905D91830E
:10150000822F0E94F50C805D808308959C01FB0171
:1015100097FD02C040E004C0309521953F4F41E067
:101520001082319780919A01DF011197882311F47D
:1015300083E401C086E4808380E28C93FD013197CF
:101540002115310519F480E3808317C0C9016AE0D1
:1015500070E00E94010D805D80833197C9016AE0CF
:1015600070E00E94010D9B016115710579F744231C
:1015700019F08DE2808331973196CF010895109252
:101580009501089510929701089581E08093990143
:10159000809198018F5F8093980148E951E061E064
:1015A00081E80E94BE08809198010895DF93CF934F
:1015B000CDB7DEB72A970FB6F894DEBF0FBECDBF0A
:1015C0000E940C0680919A010E945F0CBE01655F2B
:1015D0007F4F0E94860ADC010D900020E9F71197E9
:1015E000A81BB90BAC016A2F80E80E94BE080E94BC
:1015F0000F062A960FB6F894DEBF0FBECDBFCF916F
:10160000DF910895FC018081882319F010929701E1
:1016100003C081E0809397010E94D60A089510923A
:10162000960180E50E942D0380ED0E942D0382EE3D
:101630000E942D030E94EC020895CF93DF938091C6
:101640009A010E945F0CEC0180919A01882329F491
:1016500080E50E942D0380ED04C080ED0E942D03E3
:1016600080E50E94170305B607FE04C082EE0E94C3
:101670002D0303C082EE0E94170361E0CE010E9499
:10168000A604DF91CF910895FC018081882319F091
:1016900010929A0103C081E080939A0181E08093C7
:1016A00096010E941D0B08951F93FC011FB7F8942B
:1016B0008081882371F085B7806885BF85B7806891
:1016C00085BF0E944D0CF999FECF12BC11BC8FEF63
:1016D0000BC085B78F7785BF85B78F7785BFF999A1
:1016E000FECF12BC11BC81E080BD0FB6F894FA9A0F
:1016F000F99A0FBE1FBF1F910895DF93CF930F92EA
:10170000CDB7DEB7F999FECF12BC11BCF89A80B5FF
:101710009E012F5F3F4F8F3F19F481E0898301C005
:101720001982C9010E94540B0F90CF91DF91089547
:1017300081E0809395011092980110929B0160E0E6
:1017400081E10E94120661E081E10E94120662E0DE
:1017500081E10E94120663E081E10E9412060E946C
:10176000C50A10928500109284000895DF93CF93EC
:1017700000D0CDB7DEB79A8389830E940F0680918F
:1017800064008C60809364000E94C8020E94B502CD
:101790000E94EA0B0E94B2038FE392E00E941C06B3
:1017A00083EE0E9417030E94B8020E940F0C0E9451
:1017B0006F028823E1F70E94A602882311F00E949D
:1017C000AB02CE0101960E941C060F900F90CF91A4
:1017D000DF91089588E10FB6F8948093600010922D
:1017E00060000FBE83B7817F846083BFEC9AEBE615
:1017F000F0E080818460808383B7816083BF8895B7
:1018000083B78E7F83BFEC9808951F920F920FB617
:101810000F9211240F900FBE0F901F90189502C0C9
:101820000E94490890914301809144019817C1F7A3
:1018300088E70E948E089091430180914401981797
:10184000B9F381E00E9416090895DF93CF930F92B8
:10185000CDB7DEB76F9A779A259A90E01D9A1982D4
:1018600003C089818F5F898389818F3FD1F79F5F13
:101870009436A1F790E01D9A198203C089818F5F89
:1018800089838981803AD0F39F5F9436A1F72D98A0
:1018900077980F90CF91DF910895EEE7F0E0808187
:1018A00080618083869A8E9884988C9881E080935A
:1018B000360180E090E008951092360108951F935C
:1018C000CF93DF93182F80913601882309F43FC00E
:1018D0008E9A27E040E460E084E00E941C020E94AF
:1018E000400280E00E945302EC018FEFCF3FD80707
:1018F000C1F30E9431020E94B8028E981123B1F404
:1019000047E452E020E030E0FA01859194918C1791
:101910009D074CF02F5F3F4F4E5F5F4F2C343105DA
:1019200099F72FEF3FEF2F50304013C04FED52E0AB
:1019300020E030E0FA01859194918C179D074CF0DE
:101940002F5F3F4F4E5F5F4F2D38310599F72FEFD7
:101950003FEFC901DF91CF911F9108958DE08093F2
:10196000810084E89EE19093890080938800089527
:10197000109285001092840082E080936F00089599
:10198000EFE6F0E080818D7F808308951F920F92B3
:101990000FB60F9211248F9381E080939C018F9159
:1019A0000F900FBE0F901F901895FB01DC01059062
:1019B0000D920020E1F70895FC0105900020E9F761
:1019C000809590958E0F9F1F0895FB01DC0102C04A
:1019D00001900D9241505040D8F70895FB01DC0171
:1019E00001900D920020E1F70895991B79E004C061
:1019F000991F961708F0961B881F7A95C9F780954E
:101A0000089597FB092E07260AD077FD04D00CD045
:101A100006D000201AF4709561957F4F0895F6F76F
:101A2000909581959F4F0895AA1BBB1B51E107C05C
:101A3000AA1FBB1FA617B70710F0A61BB70B881F5E
:101A4000991F5A95A9F780959095BC01CD010895ED
:101A5000F894FFCF0100544F2020202020000000E8
:101A600000000000000000000000E299FF1C0000E0
:101A70000002000000000004000000000038040024
:101A800000A600000000000000000000001C000094
:101A900000020052020000040000000000DE04000A
:101AA00000B200000000000000000000001C000068
:101AB000000200B6040000040000000000900500D1
:101AC00000B807000000000000000000001C00003B
:101AD0000002000D140000040000000000480D008A
:101AE00000BC02000000000000000000001C00001C
:101AF00000FFFFFFFFFFFFFFFFFFFFFFFFFFFFFFF5
:101B0000FFFFFFFFFFFFFFFFFFFFFFFFFFFFFFFFE5
:101B1000FFFFFFFFFFFFFFFFFFFFFFFFFFFFFFFFD5
:101B2000FFFFFFFFFFFFFFFFFFFFFFFFFFFFFFFFC5
:101B3000FFFFFFFFFFFFFFFFFFFFFFFFFFFFFFFFB5
:108000000C94FD010C941A020C94050C0C941A02A9
:108010000C941A020C941A020C941A020C94C60CBA
:108020000C941A020C941A020C941A020C941A0260
:108030000C941A020C9496080C941A020C941A02CE
:108040000C941A020C941A020C941A020C941A0240
:108050000C941A020C941A020C94A3050C941A02A4
:108060000C941A023F065B4F666D7D077F6F777C2D
:10807000395E7971004053332944494E2E00003057
:10808000280000100800024002C593C08094199493
:108090009891881598159984809599959800000075
:1080A000000000000002020000538E9589A4B8056C
:1080B00011A4B015191509059991892020809151B5
:1080C000050111C3818385859195098595950D06D7
:1080D00014242081914103818742064220441200EA
:1080E000000000000000000000040080000080008C
:1080F0001000010100020020004000000800040000
:108100002000021000000000000000E351D1635283
:1081100062E2CDC34FCFD2ADEDF2A8A3B260E06171
:10812000E19283888DC80444D050E884C4434F4E04
:1081300054494B4900364C4F5750414E0050494E20
:10814000470050494E47494E470054454D50004D59
:108150004F444520004445472046004445472043BE
:108160000053454E44004F4E4345004155544F0087
:10817000444542554700444247204F4E0044424741
:10818000204F46460053454E540053454E44494EF9
:1081900047002D0100020000000000003501000230
:1081A0000000000000003D0100030B040000980BDC
:1081B000420102020202000000004A010005020B17
:1081C000000000004F0104060808000000005501EF
:1081D000050507070100440B5B01050506060000C5
:1081E000440B610104090505000000006601080E4A
:1081F0000A0A0000020B6B01080F09090100020BBB
:108200007001000C04020000000076010B0B0D0D44
:108210000100540B7D010B0B0C0C0000540B85016D
:10822000090E0E0E000000008A010A0F0F0F000059
:10823000000050494E4753204641494C45440057A1
:10824000414B452D2D2D009B0395038F0388038201
:10825000037B0373036C0364035C0353034B03420C
:108260000339032F0326031C0312030703FD02F245
:1082700002E702DC02D002C502B902AD02A10295FA
:108280000289027C027002630257024A023E0232F5
:1082900002250219020C020002F401E801DC01D0FF
:1082A00001C401B801AD01A20196018C01810176E2
:1082B000016C01620158014E0144013B0132012968
:1082C00001200117010F010701FF00F700F000E98D
:1082D00000E100DB00D400CD00C700C100BB00AA54
:1082E00003A703A403A1039E039B03980394039194
:1082F000038D038A03860382037E037B0377037265
:10830000036E036A03660361035D03580353034F5F
:10831000034A03450340033B03360330032B032684
:108320000320031B0315030F030A030403FE02F8D3
:1083300002F202EC02E602DF02D902D302CC02C64C
:1083400002BF02B902B202AC02A5029E02970291DC
:10835000028A0283027C0275026E02680261025A7E
:108360000253024C0245023E023702300229022229
:10837000021B0215020E0207020002F901F201ECD3
:1083800001E501DE01D801D101CB01C401BE01B775
:1083900001B101AA01A4019E01980192018C0186FC
:1083A0000180017A0174016E01680163015D015869
:1083B0000152014D01470142013D01380133012EB7
:1083C00001290124011F011A01150111010C0108E5
:1083D000010301FF00FB00F600F200EE00EA00E6F8
:1083E00000E200DE00DB00D700D300CF00CC00C8E5
:1083F00000C500C200BE00BB000011241FBECFEFAD
:10840000D8E0DEBFCDBF11E0A0E0B1E0E4E5FAE1E5
:1084100002C005900D92A631B107D9F711E0A6E18F
:10842000B1E001C01D92AD39B107E1F70E94050727
:108430000C94280D0C940000E4E6F0E090819E7FFF
:108440009083206820937A00482B40937C006093AF
:108450007B0081E0809316011092170180E090E08C
:108460000895EAE7F0E080818F778083E4E6F0E02A
:108470008081816080831092160110921701089507
:1084800080911601882319F42FEF3FEF0AC081E095
:108490008093170180917A00806480937A0020E0B5
:1084A00030E0C9010895982F80911701882399F031
:1084B00080917A0086FD0FC01092170180917C0098
:1084C0009295990F907E892B80937C002091780063
:1084D0003091790002C02FEF3FEFC90108950E944B
:1084E000400280E00E9453022FEF8F3F9207C9F3B2
:1084F000629902C080E10895803A910514F481E008
:10850000089521E08038920714F488E0089522E06D
:108510008038920714F484E008958058934014F052
:1085200080E0089582E008950E946F0290913501E5
:10853000882329F4903249F410923501089590323D
:1085400011F480E008958093350108950E9494020B
:10855000811181E008950E94A6028823E1F38091B1
:10856000350190E29093350108950E9431020895FB
:10857000EEE7F0E08081826080836A98729A819849
:10858000899827E040E460E081E00E941C020895A1
:108590008091E40084FFFCCF81E98093E400809126
:1085A000E40084FFFCCF1092E400809164008061BD
:1085B000809364000895482F6AE00E94F50C282FEC
:1085C00030E084E0220F331F8A95E1F7842F0E9468
:1085D000F50C892F822B089560E070E021C0FA012C
:1085E0008491E82FF0E0EF71F070E451FF4F2081AB
:1085F00082958695877090E0032E02C0880F991FA0
:108600000A94E2F78095822380834F5F5F4FF0E00A
:108610004D375F0721F76E5F7F4F6830710521F09E
:10862000362F46E750E0DBCF80E090E00895382F0A
:10863000E82FEF71E43180F4F0E0E451FF4F208146
:1086400032953695377081E090E002C0880F991F0F
:108650003A95E2F7282B20830895382FE82FEF7101
:10866000E43188F4F0E0E451FF4F208132953695F3
:10867000377081E090E002C0880F991F3A95E2F7C9
:1086800080958223808308950F931F93CF93DF9368
:108690009C01CB01820F931F839724F062E270E06C
:1086A000621B730BD901A55FBE4FA901620F731F37
:1086B000C1E0D0E018C0FD018491E82FEF71E431F2
:1086C00078F4F0E0E451FF4F208182958695877021
:1086D0008E0102C0000F111F8A95E2F7202B208324
:1086E0004F5F5F4F1196461757072CF3DF91CF91DD
:1086F0001F910F9108950F931F93CF93DF939C01C8
:10870000CB01820F931F839724F062E270E0621B1B
:10871000730BD901A55FBE4FA901C1E0D0E01AC01B
:10872000FD018491E82FEF71E43188F4F0E0E45129
:10873000FF4F20818295869587708E0102C0000FC1
:10874000111F8A95E2F7C8018095822380834F5FCD
:108750005F4F1196461757071CF3DF91CF911F917A
:108760000F910895809164008F7E809364008FEF55
:108770008093E50087E08093E6008EE68093E70033
:1087800088EC8093E40062E270E080E090E00E9478
:108790007B0380E290E024E0959587952A95E1F7A8
:1087A000009711F481E090E09093340180933301BD
:1087B000909332018093310180E090E00895CF934F
:1087C000DF93660F771FA6E7B0E040E050E0C82FC8
:1087D000D0E0CE01042E02C0959587950A94E2F769
:1087E00080FF16C0FD018491E82FF0E0EF71F0707A
:1087F000E451FF4F208182958695877090E0062E88
:1088000002C0880F991F0A94E2F7282B208316C014
:10881000FD018491E82FF0E0EF71F070E451FF4F1B
:10882000208182958695877090E0062E02C0880F81
:10883000991F0A94E2F78095822380834F5F5F4FF0
:1088400011964730510509F0C4CFDF91CF910895BB
:10885000AF92BF92CF92DF92EF92FF920F931F934E
:10886000CF93DF937C01C62ED42EC0E0D0E000E091
:1088700010E04FE0A42EB12CF501002E02C0EE0F47
:10888000FF1F0A94E2F7EE21FF21002E02C0F695A9
:10889000E7950A94E2F7EC59FF4FE491BE018E2F61
:1088A0000E94DF032196C430D105C1F10C5F1F4F38
:1088B000C701002E02C0969587950A94E2F7892B8E
:1088C000D9F6BE01CC2089F02196DD2019F0E5E72C
:1088D000F0E002C0E4E6F0E084910E94DF03DD20D6
:1088E000C9F48091F400806803C08091F4008F7710
:1088F0008093F4000FC0DD2019F0E4E7F0E002C03F
:10890000E4E6F0E08E010F5F1F4F8491BE010E94EC
:10891000DF03E801C430D10574F30BC0CC2021F093
:108920008091F400806803C08091F4008F77809379
:10893000F40080E090E0DF91CF911F910F91FF90C4
:10894000EF90DF90CF90BF90AF900895462F28ED25
:10895000813F920714F481EF98EDFC0187E2E0314A
:10896000F80714F0EFE0F7E2DF01F7FF04C0AA27F1
:10897000BB27AE1BBF0B8A2F6AE00E94F50C282F85
:1089800030E054E0220F331F5A95E1F76F2F661F36
:108990006627661F96EF899F802D11248A0F822BF0
:1089A00090E00E9428040895462F60E00E94280469
:1089B00008950F931F93CF93DF93982F9B016830F7
:1089C00071050CF05EC08A52813520F0903209F0BA
:1089D00058C00BC0913608F09F7D903231F0892F3E
:1089E0008A52863308F04DC001C080E0E82FF0E0E5
:1089F000EE0FFF1FE358FF4F85919591A591B4911C
:108A0000EC01822F81508695A82FB0E0A451BF4F72
:108A100068E070E440E050E0890101701070FD01F1
:108A2000E40FF51FCE018F70382F962F9F7024E032
:108A3000D695C7952A95E1F784E0769567958A954E
:108A4000E1F70115110519F0292F206F06C03295A5
:108A5000307F292F2295207F2F6090818081832B6A
:108A60009223892B8083808190812823232B2923A3
:108A700020834B5F5F4F4431510589F620E030E0A1
:108A800002C02FEF3FEFC901DF91CF911F910F91EE
:108A90000895EF92FF920F931F93CF93DF937C0182
:108AA0008B01C1E0D0E005C0BE0180E20E94D90484
:108AB0002196C017D107C4F3E8010EC0F7018081E9
:108AC000882319F4BE0180E204C00894E11CF11C63
:108AD000BE010E94D9042196C830D1057CF380E004
:108AE00090E0DF91CF911F910F91FF90EF9008954B
:108AF0000F931F9300911A0110911B01F801E45E7E
:108B0000FE4F80830F5F1F4F10931B0100931A01CC
:108B1000F801E45EFE4F10828091180190911901D6
:108B200061E070E0845E9E4F0E9449051092300122
:108B3000083011051CF081E08093300180E090E066
:108B40001F910F9108951F920F920FB60F9211244B
:108B50002F933F934F935F936F937F938F939F9345
:108B6000AF93BF93EF93FF9380913001882309F473
:108B700042C080913101909132010197909332016E
:108B800080933101892BB9F5209118013091190199
:108B9000F901E45EFE4F8081882339F410921901B7
:108BA0001092180187E090E007C080910001909139
:108BB0000101009731F0019790930101809300012A
:108BC00006C02F5F3F4F3093190120931801609129
:108BD0000001709101018091180190911901845E4A
:108BE0009E4F0E94490580913301909134019093EA
:108BF000320180933101FF91EF91BF91AF919F912D
:108C00008F917F916F915F914F913F912F910F9035
:108C10000FBE0F901F901895279A2F9808952798A8
:108C20002F9A0895E4E6F0E0E80FF11DE49170E07A
:108C30008E2F0E94DF0308950F931F938C01BC01B8
:108C40008CE191E00E94D50CC8010E94DC0C8C01E3
:108C500090931B0180931A01109219011092180130
:108C600061E070E08CE191E00E94490510923001D2
:108C7000083011051CF081E08093300180E090E025
:108C80001F910F910895CF92DF92EF92FF920F9371
:108C90001F93D82EC92E5CE1E52E51E0F52E482F0A
:108CA000592FC7010E94E50C0D2D1C2D10931B019F
:108CB00000931A01109219011092180161E070E0FE
:108CC000C7010E94490510923001083011051CF0BF
:108CD00081E08093300180E090E01F910F91FF9040
:108CE000EF90DF90CF9008950F931F93182F092FC7
:108CF000682F792F8CE191E00E94EE0CE12FF02F8C
:108D0000DF010D900020E9F78D01015010400E1B8E
:108D10001F0B10931B0100931A011092190110925E
:108D2000180161E070E08CE191E00E944905109229
:108D30003001083011051CF081E08093300180E0A3
:108D400090E01F910F9108959AE0899FF0011124FE
:108D5000EE56FE4FA7E3B1E084918D93319681E00A
:108D6000A134B807C9F7089580913701909138016F
:108D700021E08D329207A1F42CE931E0A7E3B1E0C4
:108D8000F90184918D932F5F3F4FF1E0A134BF072C
:108D9000B9F780913701909138010E941C0608951F
:108DA0008553914099F422E931E0A7E3B1E0F9015C
:108DB00084918D932F5F3F4FF1E0A134BF07B9F746
:108DC00080913701909138010E941C06089580918E
:108DD0003701909138018A54914011F40E940F0B91
:108DE00080913701909138018B56914011F40E9487
:108DF000C20A80913701909138018D53914021F43E
:108E00000E94BF0A0E94EC0208951F930E94B203C1
:108E10000E94B8020E946E080E947D0B0E944D0CB9
:108E20000E94AE0C789483EE0E9417038DEE0E9490
:108E3000170322E931E0A7E3B1E0F90184918D93B2
:108E40002F5F3F4FF1E0A134BF07B9F780913701A1
:108E5000909138010E941C060E94B80C1AE0789488
:108E600080919C018823C9F110929C010E94B40654
:108E700080919601882311F00E941D0B809197012B
:108E8000882311F00E94D60A80919501882329F148
:108E900080914101843059F480919901882339F4FB
:108EA00010924101109242010E94BF0A16C08091A7
:108EB0009901882371F010929901809142018F5F8E
:108EC00080934201843049F482E392E00E941C06C0
:108ED00004C00E94C50A809341010E94A602882313
:108EE00009F48CC00E94AB02843089F1853030F4E3
:108EF000813059F0823009F07FC018C0883009F401
:108F000037C0803109F078C04AC080913B01819F11
:108F1000F0011124EE56FE4FA7E3B1E084918D934A
:108F2000319681E0A134B807C9F760C080913C0157
:108F3000819FF0011124EE56FE4FA7E3B1E084912A
:108F40008D93319681E0A134B807C9F74FC0809165
:108F50003901819FF0011124EE56FE4FA7E3B1E0E5
:108F600084918D93319681E0A134B807C9F73EC052
:108F700080913F0190914001892B89F480913A01C1
:108F8000819FF0011124EE56FE4FA7E3B1E08491DA
:108F90008D93319681E0A134B807C9F727C0E091DD
:108FA0003F01F0914001309739F180913D0190915E
:108FB0003E01099580913D0190913E01892B31F050
:108FC00080913701909138010E941C0680913A01EE
:108FD000819FF0011124EE56FE4FA7E3B1E084918A
:108FE0008D93319681E0A134B807C9F7809137019C
:108FF000909138010E941C060E94E70680E00E94C2
:1090000016092DCFFC011182818180830895DC0136
:109010009C919F5F903508F090E011968C9111978C
:10902000981731F08C91FD01E80FF11D62839C933C
:109030000895DC0111968C911197FD01E80FF11D47
:1090400092818F5F803508F080E011968C93892F94
:109050000895109243018091430180934401089543
:10906000FC019081818120E0981321E0822F0895F6
:109070008A3010F0895C0895805D0895FB0190E3CB
:1090800090838F708A3010F0895C01C0805D81838D
:10909000089520E43BE44CE450E00BC02115310579
:1090A0004105510511F49FEF17C021503040404059
:1090B00050409091430180914401981779F3809139
:1090C0004401E82FF0E0ED5BFE4F92818F5F803529
:1090D00008F080E080934401892F0895E4E6F0E0F1
:1090E00080818D7F80831092430180914301809322
:1090F00044018CE090E09093C5008093C40086E02A
:109100008093C20088E98093C10008951092C10045
:10911000E4E6F0E08081826080830895982F80915A
:10912000C00085FFFCCF9093C60008951F920F9258
:109130000FB60F9211242F938F939F93EF93FF936A
:109140002091C600909143019F5F903508F090E018
:1091500080914401981741F0E0914301F0E0ED5B0C
:10916000FE4F228390934301FF91EF919F918F9146
:109170002F910F900FBE0F901F901895982F8091F0
:10918000C00085FFFCCF81E08093C6008091C000C5
:1091900085FFFCCF6093C6008091C00085FFFCCFA7
:1091A0009093C600FA0190E009C020818091C00030
:1091B00085FFFCCF2093C6009F5F31969617A9F7D5
:1091C0008091C00085FFFCCF84E08093C6000895A5
:1091D000DF93CF93CDB7DEB764970FB6F894DEBFB9
:1091E0000FBECDBF982FDE011196E2E0F1E088E0DE
:1091F00001900D928150E1F7FE0139968CE0DF017C
:109200001D928A95E9F7BE016C5F7F4F892F0E94FE
:10921000790ACE0101960E94740664960FB6F894FE
:10922000DEBF0FBECDBFCF91DF910895DF93CF9307
:10923000CDB7DEB72D970FB6F894DEBF0FBECDBF0A
:10924000882399F49091430180914401981769F41F
:1092500047C1211531054105510511F49FEF1CC08F
:10926000215030404040504004C020E43BE44CE4F6
:1092700050E09091430180914401981751F38091FF
:109280004401E82FF0E0ED5BFE4F92818F5F803567
:1092900008F080E08093440199838981813011F046
:1092A00081E0EDC00E940C0620E43BE44CE450E079
:1092B0000BC0211531054105510511F49FEF17C071
:1092C00021503040404050409091430180914401F2
:1092D000981779F380914401E82FF0E0ED5BFE4FA1
:1092E00092818F5F803508F080E0809344019983FC
:1092F00089818F3F11F482E0C2C0898187FF2CC031
:1093000020E43BE44CE450E00BC02115310541055D
:10931000510511F49FEF17C021503040404050409C
:109320009091430180914401981779F38091440111
:10933000E82FF0E0ED5BFE4F92818F5F803508F003
:1093400080E08093440199838981843009F4C6C008
:1093500083E00E94E808C2C089818A838A818B30B9
:1093600008F0BEC020E43BE44CE450E00BC0211503
:1093700031054105510511F49FEF17C021503040D0
:10938000404050409091430180914401981779F3F7
:1093900080914401E82FF0E0ED5BFE4F92818F5FFA
:1093A000803508F080E080934401998389818F3F64
:1093B00011F485E064C089818B8360E070E0DE0198
:1093C00014962BC0211531054105510511F49FEF6D
:1093D00017C021503040404050409091430180914F
:1093E0004401981779F380914401E82FF0E0ED5B98
:1093F000FE4F92818F5F803508F080E080934401BA
:10940000998389818F3F11F4862F39C08981FD01AD
:10941000E60FF71F80836F5F7F4F8A8190E06817A8
:10942000790728F020E43BE44CE450E010C020E44D
:109430003BE44CE450E0D1CF211531054105510505
:1094400011F49FEF17C021503040404050409091A0
:10945000430180914401981779F380914401E82FEA
:10946000F0E0ED5BFE4F92818F5F803508F080E089
:109470008093440199838981843021F087E00E94A0
:10948000E8082EC08B81813CD1F0823C09F1803C00
:1094900029F58C8180939B01813011F463E00BC02E
:1094A000823011F462E007C0833011F461E003C040
:1094B000843019F460E00E9412061092990181E54F
:1094C0000E9417030E94250C81E50E942D0306C00F
:1094D000CE0104960E9474060E94250C0E940F067D
:1094E0002D960FB6F894DEBF0FBECDBFCF91DF91A2
:1094F0000895282FFB016AE00E94F50C905D91838E
:10950000822F0E94F50C805D808308959C01FB01F1
:1095100097FD02C040E004C0309521953F4F41E0E7
:109520001082319780919A01DF011197882311F4FD
:1095300083E401C086E4808380E28C93FD0131974F
:109540002115310519F480E3808317C0C9016AE051
:1095500070E00E94010D805D80833197C9016AE04F
:1095600070E00E94010D9B016115710579F744239C
:1095700019F08DE2808331973196CF0108951092D2
:109580009501089510929701089581E080939901C3
:10959000809198018F5F8093980148E951E061E0E4
:1095A00081E80E94BE08809198010895DF93CF93CF
:1095B000CDB7DEB72A970FB6F894DEBF0FBECDBF8A
:1095C0000E940C0680919A010E945F0CBE01655FAB
:1095D0007F4F0E94860ADC010D900020E9F7119769
:1095E000A81BB90BAC016A2F80E80E94BE080E943C
:1095F0000F062A960FB6F894DEBF0FBECDBFCF91EF
:10960000DF910895FC018081882319F01092970161
:1096100003C081E0809397010E94D60A08951092BA
:10962000960180E50E942D0380ED0E942D0382EEBD
:109630000E942D030E94EC020895CF93DF93809146
:109640009A010E945F0CEC0180919A01882329F411
:1096500080E50E942D0380ED04C080ED0E942D0363
:1096600080E50E94170305B607FE04C082EE0E9443
:109670002D0303C082EE0E94170361E0CE010E9419
:10968000A604DF91CF910895FC018081882319F011
:1096900010929A0103C081E080939A0181E0809347
:1096A00096010E941D0B08951F93FC011FB7F894AB
:1096B0008081882371F085B7806885BF85B7806811
:1096C00085BF0E944D0CF999FECF12BC11BC8FEFE3
:1096D0000BC085B78F7785BF85B78F7785BFF99921
:1096E000FECF12BC11BC81E080BD0FB6F894FA9A8F
:1096F000F99A0FBE1FBF1F910895DF93CF930F926A
:10970000CDB7DEB7F999FECF12BC11BCF89A80B57F
:109710009E012F5F3F4F8F3F19F481E0898301C085
:109720001982C9010E94540B0F90CF91DF910895C7
:1097300081E0809395011092980110929B0160E066
:1097400081E10E94120661E081E10E94120662E05E
:1097500081E10E94120663E081E10E9412060E94EC
:10976000C50A10928500109284000895DF93CF936C
:1097700000D0CDB7DEB79A8389830E940F0680910F
:1097800064008C60809364000E94C8020E94B5024D
:109790000E94EA0B0E94B2038FE392E00E941C0633
:1097A00083EE0E9417030E94B8020E940F0C0E94D1
:1097B0006F028823E1F70E94A602882311F00E941D
:1097C000AB02CE0101960E941C060F900F90CF9124
:1097D000DF91089588E10FB6F894809360001092AD
:1097E00060000FBE83B7817F846083BFEC9AEBE695
:1097F000F0E080818460808383B7816083BF889537
:1098000083B78E7F83BFEC9808951F920F920FB697
:109810000F9211240F900FBE0F901F90189502C049
:109820000E94490890914301809144019817C1F723
:1098300088E70E948E089091430180914401981717
:10984000B9F381E00E9416090895DF93CF930F9238
:10985000CDB7DEB76F9A779A259A90E01D9A198254
:1098600003C089818F5F898389818F3FD1F79F5F93
:109870009436A1F790E01D9A198203C089818F5F09
:1098800089838981803AD0F39F5F9436A1F72D9820
:1098900077980F90CF91DF910895EEE7F0E0808107
:1098A00080618083869A8E9884988C9881E08093DA
:1098B000360180E090E008951092360108951F93DC
:1098C000CF93DF93182F80913601882309F43FC08E
:1098D0008E9A27E040E460E084E00E941C020E942F
:1098E000400280E00E945302EC018FEFCF3FD80787
:1098F000C1F30E9431020E94B8028E981123B1F484
:1099000047E452E020E030E0FA01859194918C1711
:109910009D074CF02F5F3F4F4E5F5F4F2C3431055A
:1099200099F72FEF3FEF2F50304013C04FED52E02B
:1099300020E030E0FA01859194918C179D074CF05E
:109940002F5F3F4F4E5F5F4F2D38310599F72FEF57
:109950003FEFC901DF91CF911F9108958DE0809372
:10996000810084E89EE190938900809388000895A7
:10997000109285001092840082E080936F00089519
:10998000EFE6F0E080818D7F808308951F920F9233
:109990000FB60F9211248F9381E080939C018F91D9
:1099A0000F900FBE0F901F901895FB01DC010590E2
:1099B0000D920020E1F70895FC0105900020E9F7E1
:1099C000809590958E0F9F1F0895FB01DC0102C0CA
:1099D00001900D9241505040D8F70895FB01DC01F1
:1099E00001900D920020E1F70895991B79E004C0E1
:1099F000991F961708F0961B881F7A95C9F78095CE
:109A0000089597FB092E07260AD077FD04D00CD0C5
:109A100006D000201AF4709561957F4F0895F6F7EF
:109A2000909581959F4F0895AA1BBB1B51E107C0DC
:109A3000AA1FBB1FA617B70710F0A61BB70B881FDE
:109A4000991F5A95A9F780959095BC01CD0108956D
:109A5000F894FFCF0100544F202020202000000068
:109A600000000000000000000000E299FF1C000060
:109A700000020000000000040000000000380400A4
:109A800000A600000000000000000000001C000014
:109A900000020052020000040000000000DE04008A
:109AA00000B200000000000000000000001C0000E8
:109AB000000200B604000004000000000090050051
:109AC00000B807000000000000000000001C0000BB
:109AD0000002000D140000040000000000480D000A
:109AE00000BC02000000000000000000001C00009C
:109AF00000FFFFFFFFFFFFFFFFFFFFFFFFFFFFFF75
:109B0000FFFFFFFFFFFFFFFFFFFFFFFFFFFFFFFF65
:109B1000FFFFFFFFFFFFFFFFFFFFFFFFFFFFFFFF55
:109B2000FFFFFFFFFFFFFFFFFFFFFFFFFFFFFFFF45
:109B3000FFFFFFFFFFFFFFFFFFFFFFFFFFFFFFFF35
:020000021000EC
:100000000C94FD010C941A020C94050C0C941A0229
:100010000C941A020C941A020C941A020C94C60C3A
:100020000C941A020C941A020C941A020C941A02E0
:100030000C941A020C9496080C941A020C941A024E
:100040000C941A020C941A020C941A020C941A02C0
:100050000C941A020C941A020C94A3050C941A0224
:100060000C941A023F065B4F666D7D077F6F777CAD
:10007000395E7971004053332944494E2E000030D7
:10008000280000100800024002C593C08094199413
:1000900098918815981599848095999598000000F5
:1000A000000000000002020000538E9589A4B805EC
:1000B00011A4B01519150905999189202080915135
:1000C000050111C3818385859195098595950D0657
:1000D000142420819141038187420642204412006A
:1000E000000000000000000000040080000080000C
:1000F0001000010100020020004000000800040080
:100100002000021000000000000000E351D1635203
:1001100062E2CDC34FCFD2ADEDF2A8A3B260E061F1
:10012000E19283888DC80444D050E884C4434F4E84
:1001300054494B4900364C4F5750414E0050494EA0
:10014000470050494E47494E470054454D50004DD9
:100150004F4445200044454720460044454720433E
:100160000053454E44004F4E4345004155544F0007
:10017000444542554700444247204F4E00444247C1
:10018000204F46460053454E540053454E44494E79
:1001900047002D01000200000000000035010002B0
:1001A0000000000000003D0100030B040000980B5C
:1001B000420102020202000000004A010005020B97
:1001C000000000004F01040608080000000055016F
:1001D000050507070100440B5B0105050606000045
:1001E000440B610104090505000000006601080ECA
:1001F0000A0A0000020B6B01080F09090100020B3B
:100200007001000C04020000000076010B0B0D0DC4
:100210000100540B7D010B0B0C0C0000540B8501ED
:10022000090E0E0E000000008A010A0F0F0F0000D9
:10023000000050494E4753204641494C4544005721
:10024000414B452D2D2D009B0395038F0388038281
:10025000037B0373036C0364035C0353034B03428C
:100260000339032F0326031C0312030703FD02F2C5
:1002700002E702DC02D002C502B902AD02A102957A
:100280000289027C027002630257024A023E023275
:1002900002250219020C020002F401E801DC01D07F
:1002A00001C401B801AD01A20196018C0181017662
:1002B000016C01620158014E0144013B01320129E8
:1002C00001200117010F010701FF00F700F000E90D
:1002D00000E100DB00D400CD00C700C100BB00AAD4
:1002E00003A703A403A1039E039B03980394039114
:1002F000038D038A03860382037E037B03770372E5
:10030000036E036A03660361035D03580353034FDF
:10031000034A03450340033B03360330032B032604
:100320000320031B0315030F030A030403FE02F853
:1003300002F202EC02E602DF02D902D302CC02C6CC
:1003400002BF02B902B202AC02A5029E029702915C
:10035000028A0283027C0275026E02680261025AFE
:100360000253024C0245023E0237023002290222A9
:10037000021B0215020E0207020002F901F201EC53
:1003800001E501DE01D801D101CB01C401BE01B7F5
:1003900001B101AA01A4019E01980192018C01867C
:1003A0000180017A0174016E01680163015D0158E9
:1003B0000152014D01470142013D01380133012E37
:1003C00001290124011F011A01150111010C010865
:1003D000010301FF00FB00F600F200EE00EA00E678
:1003E00000E200DE00DB00D700D300CF00CC00C865
:1003F00000C500C200BE00BB000011241FBECFEF2D
:10040000D8E0DEBFCDBF11E0A0E0B1E0E4E5FAE165
:1004100002C005900D92A631B107D9F711E0A6E10F
:10042000B1E001C01D92AD39B107E1F70E940507A7
:100430000C94280D0C940000E4E6F0E090819E7F7F
:100440009083206820937A00482B40937C0060932F
:100450007B0081E0809316011092170180E090E00C
:100460000895EAE7F0E080818F778083E4E6F0E0AA
:100470008081816080831092160110921701089587
:1004800080911601882319F42FEF3FEF0AC081E015
:100490008093170180917A00806480937A0020E035
:1004A00030E0C9010895982F80911701882399F0B1
:1004B00080917A0086FD0FC01092170180917C0018
:1004C0009295990F907E892B80937C0020917800E3
:1004D0003091790002C02FEF3FEFC90108950E94CB
:1004E000400280E00E9453022FEF8F3F9207C9F332
:1004F000629902C080E10895803A910514F481E088
:10050000089521E08038920714F488E0089522E0ED
:100510008038920714F484E008958058934014F0D2
:1005200080E0089582E008950E946F029091350165
:10053000882329F4903249F41092350108959032BD
:1005400011F480E008958093350108950E9494028B
:10055000811181E008950E94A6028823E1F3809131
:10056000350190E29093350108950E94310208957B
:10057000EEE7F0E08081826080836A98729A8198C9
:10058000899827E040E460E081E00E941C02089521
:100590008091E40084FFFCCF81E98093E4008091A6
:1005A000E40084FFFCCF1092E4008091640080613D
:1005B000809364000895482F6AE00E94F50C282F6C
:1005C00030E084E0220F331F8A95E1F7842F0E94E8
:1005D000F50C892F822B089560E070E021C0FA01AC
:1005E0008491E82FF0E0EF71F070E451FF4F20812B
:1005F00082958695877090E0032E02C0880F991F20
:100600000A94E2F78095822380834F5F5F4FF0E08A
:100610004D375F0721F76E5F7F4F6830710521F01E
:10062000362F46E750E0DBCF80E090E00895382F8A
:10063000E82FEF71E43180F4F0E0E451FF4F2081C6
:1006400032953695377081E090E002C0880F991F8F
:100650003A95E2F7282B20830895382FE82FEF7181
:10066000E43188F4F0E0E451FF4F20813295369573
:10067000377081E090E002C0880F991F3A95E2F749
:1006800080958223808308950F931F93CF93DF93E8
:100690009C01CB01820F931F839724F062E270E0EC
:1006A000621B730BD901A55FBE4FA901620F731FB7
:1006B000C1E0D0E018C0FD018491E82FEF71E43172
:1006C00078F4F0E0E451FF4F2081829586958770A1
:1006D0008E0102C0000F111F8A95E2F7202B2083A4
:1006E0004F5F5F4F1196461757072CF3DF91CF915D
:1006F0001F910F9108950F931F93CF93DF939C0148
:10070000CB01820F931F839724F062E270E0621B9B
:10071000730BD901A55FBE4FA901C1E0D0E01AC09B
:10072000FD018491E82FEF71E43188F4F0E0E451A9
:10073000FF4F20818295869587708E0102C0000F41
:10074000111F8A95E2F7C8018095822380834F5F4D
:100750005F4F1196461757071CF3DF91CF911F91FA
:100760000F910895809164008F7E809364008FEFD5
:100770008093E50087E08093E6008EE68093E700B3
:1007800088EC8093E40062E270E080E090E00E94F8
:100790007B0380E290E024E0959587952A95E1F728
:1007A000009711F481E090E090933401809333013D
:1007B000909332018093310180E090E00895CF93CF
:1007C000DF93660F771FA6E7B0E040E050E0C82F48
:1007D000D0E0CE01042E02C0959587950A94E2F7E9
:1007E00080FF16C0FD018491E82FF0E0EF71F070FA
:1007F000E451FF4F208182958695877090E0062E08
:1008000002C0880F991F0A94E2F7282B208316C094
:10081000FD018491E82FF0E0EF71F070E451FF4F9B
:10082000208182958695877090E0062E02C0880F01
:10083000991F0A94E2F78095822380834F5F5F4F70
:1008400011964730510509F0C4CFDF91CF9108953B
:10085000AF92BF92CF92DF92EF92FF920F931F93CE
:10086000CF93DF937C01C62ED42EC0E0D0E000E011
:1008700010E04FE0A42EB12CF501002E02C0EE0FC7
:10088000FF1F0A94E2F7EE21FF21002E02C0F69529
:10089000E7950A94E2F7EC59FF4FE491BE018E2FE1
:1008A0000E94DF032196C430D105C1F10C5F1F4FB8
:1008B000C701002E02C0969587950A94E2F7892B0E
:1008C000D9F6BE01CC2089F02196DD2019F0E5E7AC
:1008D000F0E002C0E4E6F0E084910E94DF03DD2056
:1008E000C9F48091F400806803C08091F4008F7790
:1008F0008093F4000FC0DD2019F0E4E7F0E002C0BF
:10090000E4E6F0E08E010F5F1F4F8491BE010E946C
:10091000DF03E801C430D10574F30BC0CC2021F013
:100920008091F400806803C08091F4008F778093F9
:10093000F40080E090E0DF91CF911F910F91FF9044
:10094000EF90DF90CF90BF90AF900895462F28EDA5
:10095000813F920714F481EF98EDFC0187E2E031CA
:10096000F80714F0EFE0F7E2DF01F7FF04C0AA2771
:10097000BB27AE1BBF0B8A2F6AE00E94F50C282F05
:1009800030E054E0220F331F5A95E1F76F2F661FB6
:100990006627661F96EF899F802D11248A0F822B70
:1009A00090E00E9428040895462F60E00E942804E9
:1009B00008950F931F93CF93DF93982F9B01683077
:1009C00071050CF05EC08A52813520F0903209F03A
:1009D00058C00BC0913608F09F7D903231F0892FBE
:1009E0008A52863308F04DC001C080E0E82FF0E065
:1009F000EE0FFF1FE358FF4F85919591A591B4919C
:100A0000EC01822F81508695A82FB0E0A451BF4FF2
:100A100068E070E440E050E0890101701070FD0171
:100A2000E40FF51FCE018F70382F962F9F7024E0B2
:100A3000D695C7952A95E1F784E0769567958A95CE
:100A4000E1F70115110519F0292F206F06C0329525
:100A5000307F292F2295207F2F6090818081832BEA
:100A60009223892B8083808190812823232B292323
:100A700020834B5F5F4F4431510589F620E030E021
:100A800002C02FEF3FEFC901DF91CF911F910F916E
:100A90000895EF92FF920F931F93CF93DF937C0102
:100AA0008B01C1E0D0E005C0BE0180E20E94D90404
:100AB0002196C017D107C4F3E8010EC0F701808169
:100AC000882319F4BE0180E204C00894E11CF11CE3
:100AD000BE010E94D9042196C830D1057CF380E084
:100AE00090E0DF91CF911F910F91FF90EF900895CB
:100AF0000F931F9300911A0110911B01F801E45EFE
:100B0000FE4F80830F5F1F4F10931B0100931A014C
:100B1000F801E45EFE4F1082809118019091190156
:100B200061E070E0845E9E4F0E94490510923001A2
:100B3000083011051CF081E08093300180E090E0E6
:100B40001F910F9108951F920F920FB60F921124CB
:100B50002F933F934F935F936F937F938F939F93C5
:100B6000AF93BF93EF93FF9380913001882309F4F3
:100B700042C08091310190913201019790933201EE
:100B800080933101892BB9F5209118013091190119
:100B9000F901E45EFE4F8081882339F41092190137
:100BA0001092180187E090E007C0809100019091B9
:100BB0000101009731F001979093010180930001AA
:100BC00006C02F5F3F4F30931901209318016091A9
:100BD0000001709101018091180190911901845ECA
:100BE0009E4F0E944905809133019091340190936A
:100BF000320180933101FF91EF91BF91AF919F91AD
:100C00008F917F916F915F914F913F912F910F90B5
:100C10000FBE0F901F901895279A2F980895279828
:100C20002F9A0895E4E6F0E0E80FF11DE49170E0FA
:100C30008E2F0E94DF0308950F931F938C01BC0138
:100C40008CE191E00E94D50CC8010E94DC0C8C0163
:100C500090931B0180931A011092190110921801B0
:100C600061E070E08CE191E00E9449051092300152
:100C7000083011051CF081E08093300180E090E0A5
:100C80001F910F910895CF92DF92EF92FF920F93F1
:100C90001F93D82EC92E5CE1E52E51E0F52E482F8A
:100CA000592FC7010E94E50C0D2D1C2D10931B011F
:100CB00000931A01109219011092180161E070E07E
:100CC000C7010E94490510923001083011051CF03F
:100CD00081E08093300180E090E01F910F91FF90C0
:100CE000EF90DF90CF9008950F931F93182F092F47
:100CF000682F792F8CE191E00E94EE0CE12FF02F0C
:100D0000DF010D900020E9F78D01015010400E1B0E
:100D10001F0B10931B0100931A01109219011092DE
:100D2000180161E070E08CE191E00E9449051092A9
:100D30003001083011051CF081E08093300180E023
:100D400090E01F910F9108959AE0899FF00111247E
:100D5000EE56FE4FA7E3B1E084918D93319681E08A
:100D6000A134B807C9F708958091370190913801EF
:100D700021E08D329207A1F42CE931E0A7E3B1E044
:100D8000F90184918D932F5F3F4FF1E0A134BF07AC
:100D9000B9F780913701909138010E941C0608959F
:100DA0008553914099F422E931E0A7E3B1E0F901DC
:100DB00084918D932F5F3F4FF1E0A134BF07B9F7C6
:100DC00080913701909138010E941C06089580910E
:100DD0003701909138018A54914011F40E940F0B11
:100DE00080913701909138018B56914011F40E9407
:100DF000C20A80913701909138018D53914021F4BE
:100E00000E94BF0A0E94EC0208951F930E94B20341
:100E10000E94B8020E946E080E947D0B0E944D0C39
:100E20000E94AE0C789483EE0E9417038DEE0E9410
:100E3000170322E931E0A7E3B1E0F90184918D9332
:100E40002F5F3F4FF1E0A134BF07B9F78091370121
:100E5000909138010E941C060E94B80C1AE0789408
:100E600080919C018823C9F110929C010E94B406D4
:100E700080919601882311F00E941D0B80919701AB
:100E8000882311F00E94D60A80919501882329F1C8
:100E900080914101843059F480919901882339F47B
:100EA00010924101109242010E94BF0A16C0809127
:100EB0009901882371F010929901809142018F5F0E
:100EC00080934201843049F482E392E00E941C0640
:100ED00004C00E94C50A809341010E94A602882393
:100EE00009F48CC00E94AB02843089F1853030F463
:100EF000813059F0823009F07FC018C0883009F481
:100F000037C0803109F078C04AC080913B01819F91
:100F1000F0011124EE56FE4FA7E3B1E084918D93CA
:100F2000319681E0A134B807C9F760C080913C01D7
:100F3000819FF0011124EE56FE4FA7E3B1E08491AA
:100F40008D93319681E0A134B807C9F74FC08091E5
:100F50003901819FF0011124EE56FE4FA7E3B1E065
:100F600084918D93319681E0A134B807C9F73EC0D2
:100F700080913F0190914001892B89F480913A0141
:100F8000819FF0011124EE56FE4FA7E3B1E084915A
:100F90008D93319681E0A134B807C9F727C0E0915D
:100FA0003F01F0914001309739F180913D019091DE
:100FB0003E01099580913D0190913E01892B31F0D0
:100FC00080913701909138010E941C0680913A016E
:100FD000819FF0011124EE56FE4FA7E3B1E084910A
:100FE0008D93319681E0A134B807C9F7809137011C
:100FF000909138010E941C060E94E70680E00E9442
:1010000016092DCFFC011182818180830895DC01B6
:101010009C919F5F903508F090E011968C9111970C
:10102000981731F08C91FD01E80FF11D62839C93BC
:101030000895DC0111968C911197FD01E80FF11DC7
:1010400092818F5F803508F080E011968C93892F14
:1010500008951092430180914301809344010895C3
:10106000FC019081818120E0981321E0822F089576
:101070008A3010F0895C0895805D0895FB0190E34B
:1010800090838F708A3010F0895C01C0805D81830D
:10109000089520E43BE44CE450E00BC021153105F9
:1010A0004105510511F49FEF17C0215030404040D9
:1010B00050409091430180914401981779F38091B9
:1010C0004401E82FF0E0ED5BFE4F92818F5F8035A9
:1010D00008F080E080934401892F0895E4E6F0E071
:1010E00080818D7F808310924301809143018093A2
:1010F00044018CE090E09093C5008093C40086E0AA
:101100008093C20088E98093C10008951092C100C5
:10111000E4E6F0E08081826080830895982F8091DA
:10112000C00085FFFCCF9093C60008951F920F92D8
:101130000FB60F9211242F938F939F93EF93FF93EA
:101140002091C600909143019F5F903508F090E098
:1011500080914401981741F0E0914301F0E0ED5B8C
:10116000FE4F228390934301FF91EF919F918F91C6
:101170002F910F900FBE0F901F901895982F809170
:10118000C00085FFFCCF81E08093C6008091C00045
:1011900085FFFCCF6093C6008091C00085FFFCCF27
:1011A0009093C600FA0190E009C020818091C000B0
:1011B00085FFFCCF2093C6009F5F31969617A9F755
:1011C0008091C00085FFFCCF84E08093C600089525
:1011D000DF93CF93CDB7DEB764970FB6F894DEBF39
:1011E0000FBECDBF982FDE011196E2E0F1E088E05E
:1011F00001900D928150E1F7FE0139968CE0DF01FC
:101200001D928A95E9F7BE016C5F7F4F892F0E947E
:10121000790ACE0101960E94740664960FB6F8947E
:10122000DEBF0FBECDBFCF91DF910895DF93CF9387
:10123000CDB7DEB72D970FB6F894DEBF0FBECDBF8A
:10124000882399F49091430180914401981769F49F
:1012500047C1211531054105510511F49FEF1CC00F
:10126000215030404040504004C020E43BE44CE476
:1012700050E09091430180914401981751F380917F
:101280004401E82FF0E0ED5BFE4F92818F5F8035E7
:1012900008F080E08093440199838981813011F0C6
:1012A00081E0EDC00E940C0620E43BE44CE450E0F9
:1012B0000BC0211531054105510511F49FEF17C0F1
:1012C0002150304040405040909143018091440172
:1012D000981779F380914401E82FF0E0ED5BFE4F21
:1012E00092818F5F803508F080E08093440199837C
:1012F00089818F3F11F482E0C2C0898187FF2CC0B1
:1013000020E43BE44CE450E00BC0211531054105DD
:10131000510511F49FEF17C021503040404050401C
:101320009091430180914401981779F38091440191
:10133000E82FF0E0ED5BFE4F92818F5F803508F083
:1013400080E08093440199838981843009F4C6C088
:1013500083E00E94E808C2C089818A838A818B3039
:1013600008F0BEC020E43BE44CE450E00BC0211583
:1013700031054105510511F49FEF17C02150304050
:10138000404050409091430180914401981779F377
:1013900080914401E82FF0E0ED5BFE4F92818F5F7A
:1013A000803508F080E080934401998389818F3FE4
:1013B00011F485E064C089818B8360E070E0DE0118
:1013C00014962BC0211531054105510511F49FEFED
:1013D00017C02150304040405040909143018091CF
:1013E0004401981779F380914401E82FF0E0ED5B18
:1013F000FE4F92818F5F803508F080E0809344013A
:10140000998389818F3F11F4862F39C08981FD012D
:10141000E60FF71F80836F5F7F4F8A8190E0681728
:10142000790728F020E43BE44CE450E010C020E4CD
:101430003BE44CE450E0D1CF211531054105510585
:1014400011F49FEF17C02150304040405040909120
:10145000430180914401981779F380914401E82F6A
:10146000F0E0ED5BFE4F92818F5F803508F080E009
:101470008093440199838981843021F087E00E9420
:10148000E8082EC08B81813CD1F0823C09F1803C80
:1014900029F58C8180939B01813011F463E00BC0AE
:1014A000823011F462E007C0833011F461E003C0C0
:1014B000843019F460E00E9412061092990181E5CF
:1014C0000E9417030E94250C81E50E942D0306C08F
:1014D000CE0104960E9474060E94250C0E940F06FD
:1014E0002D960FB6F894DEBF0FBECDBFCF91DF9122
:1014F0000895282FFB016AE00E94F50C905D91830E
:10150000822F0E94F50C805D808308959C01FB0171
:1015100097FD02C040E004C0309521953F4F41E067
:101520001082319780919A01DF011197882311F47D
:1015300083E401C086E4808380E28C93FD013197CF
:101540002115310519F480E3808317C0C9016AE0D1
:1015500070E00E94010D805D80833197C9016AE0CF
:1015600070E00E94010D9B016115710579F744231C
:1015700019F08DE2808331973196CF010895109252
:101580009501089510929701089581E08093990143
:10159000809198018F5F8093980148E951E061E064
:1015A00081E80E94BE08809198010895DF93CF934F
:1015B000CDB7DEB72A970FB6F894DEBF0FBECDBF0A
:1015C0000E940C0680919A010E945F0CBE01655F2B
:1015D0007F4F0E94860ADC010D900020E9F71197E9
:1015E000A81BB90BAC016A2F80E80E94BE080E94BC
:1015F0000F062A960FB6F894DEBF0FBECDBFCF916F
:10160000DF910895FC018081882319F010929701E1
:1016100003C081E0809397010E94D60A089510923A
:10162000960180E50E942D0380ED0E942D0382EE3D
:101630000E942D030E94EC020895CF93DF938091C6
:101640009A010E945F0CEC0180919A01882329F491
:1016500080E50E942D0380ED04C080ED0E942D03E3
:1016600080E50E94170305B607FE04C082EE0E94C3
:101670002D0303C082EE0E94170361E0CE010E9499
:10168000A604DF91CF910895FC018081882319F091
:1016900010929A0103C081E080939A0181E08093C7
:1016A00096010E941D0B08951F93FC011FB7F8942B
:1016B0008081882371F085B7806885BF85B7806891
:1016C00085BF0E944D0CF999FECF12BC11BC8FEF63
:1016D0000BC085B78F7785BF85B78F7785BFF999A1
:1016E000FECF12BC11BC81E080BD0FB6F894FA9A0F
:1016F000F99A0FBE1FBF1F910895DF93CF930F92EA
:10170000CDB7DEB7F999FECF12BC11BCF89A80B5FF
:101710009E012F5F3F4F8F3F19F481E0898301C005
:101720001982C9010E94540B0F90CF91DF91089547
:1017300081E0809395011092980110929B0160E0E6
:1017400081E10E94120661E081E10E94120662E0DE
:1017500081E10E94120663E081E10E9412060E946C
:10176000C50A10928500109284000895DF93CF93EC
:1017700000D0CDB7DEB79A8389830E940F0680918F
:1017800064008C60809364000E94C8020E94B502CD
:101790000E94EA0B0E94B2038FE392E00E941C06B3
:1017A00083EE0E9417030E94B8020E940F0C0E9451
:1017B0006F028823E1F70E94A602882311F00E949D
:1017C000AB02CE0101960E941C060F900F90CF91A4
:1017D000DF91089588E10FB6F8948093600010922D
:1017E00060000FBE83B7817F846083BFEC9AEBE615
:1017F000F0E080818460808383B7816083BF8895B7
:1018000083B78E7F83BFEC9808951F920F920FB617
:101810000F9211240F900FBE0F901F90189502C0C9
:101820000E94490890914301809144019817C1F7A3
:1018300088E70E948E089091430180914401981797
:10184000B9F381E00E9416090895DF93CF930F92B8
:10185000CDB7DEB76F9A779A259A90E01D9A1982D4
:1018600003C089818F5F898389818F3FD1F79F5F13
:101870009436A1F790E01D9A198203C089818F5F89
:1018800089838981803AD0F39F5F9436A1F72D98A0
:1018900077980F90CF91DF910895EEE7F0E0808187
:1018A00080618083869A8E9884988C9881E080935A
:1018B000360180E090E008951092360108951F935C
:1018C000CF93DF93182F80913601882309F43FC00E
:1018D0008E9A27E040E460E084E00E941C020E94AF
:1018E000400280E00E945302EC018FEFCF3FD80707
:1018F000C1F30E9431020E94B8028E981123B1F404
:1019000047E452E020E030E0FA01859194918C1791
:101910009D074CF02F5F3F4F4E5F5F4F2C343105DA
:1019200099F72FEF3FEF2F50304013C04FED52E0AB
:1019300020E030E0FA01859194918C179D074CF0DE
:101940002F5F3F4F4E5F5F4F2D38310599F72FEFD7
:101950003FEFC901DF91CF911F9108958DE08093F2
:10196000810084E89EE19093890080938800089527
:10197000109285001092840082E080936F00089599
:10198000EFE6F0E080818D7F808308951F920F92B3
:101990000FB60F9211248F9381E080939C018F9159
:1019A0000F900FBE0F901F901895FB01DC01059062
:1019B0000D920020E1F70895FC0105900020E9F761
:1019C000809590958E0F9F1F0895FB01DC0102C04A
:1019D00001900D9241505040D8F70895FB01DC0171
:1019E00001900D920020E1F70895991B79E004C061
:1019F000991F961708F0961B881F7A95C9F780954E
:101A0000089597FB092E07260AD077FD04D00CD045
:101A100006D000201AF4709561957F4F0895F6F76F
:101A2000909581959F4F0895AA1BBB1B51E107C05C
:101A3000AA1FBB1FA617B70710F0A61BB70B881F5E
:101A4000991F5A95A9F780959095BC01CD010895ED
:101A5000F894FFCF0100544F2020202020000000E8
:101A600000000000000000000000E299FF1C0000E0
:101A70000002000000000004000000000038040024
:101A800000A600000000000000000000001C000094
:101A900000020052020000040000000000DE04000A
:101AA00000B200000000000000000000001C000068
:101AB000000200B6040000040000000000900500D1
:101AC00000B807000000000000000000001C00003B
:101AD0000002000D140000040000000000480D008A
:101AE00000BC02000000000000000000001C00001C
:101AF00000FFFFFFFFFFFFFFFFFFFFFFFFFFFFFFF5
:101B0000FFFFFFFFFFFFFFFFFFFFFFFFFFFFFFFFE5
:101B1000FFFFFFFFFFFFFFFFFFFFFFFFFFFFFFFFD5
:101B2000FFFFFFFFFFFFFFFFFFFFFFFFFFFFFFFFC5
:101B3000FFFFFFFFFFFFFFFFFFFFFFFFFFFFFFFFB5
:108000000C94FD010C941A020C94050C0C941A02A9
:108010000C941A020C941A020C941A020C94C60CBA
:108020000C941A020C941A020C941A020C941A0260
:108030000C941A020C9496080C941A020C941A02CE
:108040000C941A020C941A020C941A020C941A0240
:108050000C941A020C941A020C94A3050C941A02A4
:108060000C941A023F065B4F666D7D077F6F777C2D
:10807000395E7971004053332944494E2E00003057
:10808000280000100800024002C593C08094199493
:108090009891881598159984809599959800000075
:1080A000000000000002020000538E9589A4B8056C
:1080B00011A4B015191509059991892020809151B5
:1080C000050111C3818385859195098595950D06D7
:1080D00014242081914103818742064220441200EA
:1080E000000000000000000000040080000080008C
:1080F0001000010100020020004000000800040000
:108100002000021000000000000000E351D1635283
:1081100062E2CDC34FCFD2ADEDF2A8A3B260E06171
:10812000E19283888DC80444D050E884C4434F4E04
:1081300054494B4900364C4F5750414E0050494E20
:10814000470050494E47494E470054454D50004D59
:108150004F444520004445472046004445472043BE
:108160000053454E44004F4E4345004155544F0087
:10817000444542554700444247204F4E0044424741
:10818000204F46460053454E540053454E44494EF9
:1081900047002D0100020000000000003501000230
:1081A0000000000000003D0100030B040000980BDC
:1081B000420102020202000000004A010005020B17
:1081C000000000004F0104060808000000005501EF
:1081D000050507070100440B5B01050506060000C5
:1081E000440B610104090505000000006601080E4A
:1081F0000A0A0000020B6B01080F09090100020BBB
:108200007001000C04020000000076010B0B0D0D44
:108210000100540B7D010B0B0C0C0000540B85016D
:10822000090E0E0E000000008A010A0F0F0F000059
:10823000000050494E4753204641494C45440057A1
:10824000414B452D2D2D009B0395038F0388038201
:10825000037B0373036C0364035C0353034B03420C
:108260000339032F0326031C0312030703FD02F245
:1082700002E702DC02D002C502B902AD02A10295FA
:108280000289027C027002630257024A023E0232F5
:1082900002250219020C020002F401E801DC01D0FF
:1082A00001C401B801AD01A20196018C01810176E2
:1082B000016C01620158014E0144013B0132012968
:1082C00001200117010F010701FF00F700F000E98D
:1082D00000E100DB00D400CD00C700C100BB00AA54
:1082E00003A703A403A1039E039B03980394039194
:1082F000038D038A03860382037E037B0377037265
:10830000036E036A03660361035D03580353034F5F
:10831000034A03450340033B03360330032B032684
:108320000320031B0315030F030A030403FE02F8D3
:1083300002F202EC02E602DF02D902D302CC02C64C
:1083400002BF02B902B202AC02A5029E02970291DC
:10835000028A0283027C0275026E02680261025A7E
:108360000253024C0245023E023702300229022229
:10837000021B0215020E0207020002F901F201ECD3
:1083800001E501DE01D801D101CB01C401BE01B775
:1083900001B101AA01A4019E01980192018C0186FC
:1083A0000180017A0174016E01680163015D015869
:1083B0000152014D01470142013D01380133012EB7
:1083C00001290124011F011A01150111010C0108E5
:1083D000010301FF00FB00F600F200EE00EA00E6F8
:1083E00000E200DE00DB00D700D300CF00CC00C8E5
:1083F00000C500C200BE00BB000011241FBECFEFAD
:10840000D8E0DEBFCDBF11E0A0E0B1E0E4E5FAE1E5
:1084100002C005900D92A631B107D9F711E0A6E18F
:10842000B1E001C01D92AD39B107E1F70E94050727
:108430000C94280D0C940000E4E6F0E090819E7FFF
:108440009083206820937A00482B40937C006093AF
:108450007B0081E0809316011092170180E090E08C
:108460000895EAE7F0E080818F778083E4E6F0E02A
:108470008081816080831092160110921701089507
:1084800080911601882319F42FEF3FEF0AC081E095
:108490008093170180917A00806480937A0020E0B5
:1084A00030E0C9010895982F80911701882399F031
:1084B00080917A0086FD0FC01092170180917C0098
:1084C0009295990F907E892B80937C002091780063
:1084D0003091790002C02FEF3FEFC90108950E944B
:1084E000400280E00E9453022FEF8F3F9207C9F3B2
:1084F000629902C080E10895803A910514F481E008
:10850000089521E08038920714F488E0089522E06D
:108510008038920714F484E008958058934014F052
:1085200080E0089582E008950E946F0290913501E5
:10853000882329F4903249F410923501089590323D
:1085400011F480E008958093350108950E9494020B
:10855000811181E008950E94A6028823E1F38091B1
:10856000350190E29093350108950E9431020895FB
:10857000EEE7F0E08081826080836A98729A819849
:10858000899827E040E460E081E00E941C020895A1
:108590008091E40084FFFCCF81E98093E400809126
:1085A000E40084FFFCCF1092E400809164008061BD
:1085B000809364000895482F6AE00E94F50C282FEC
:1085C00030E084E0220F331F8A95E1F7842F0E9468
:1085D000F50C892F822B089560E070E021C0FA012C
:1085E0008491E82FF0E0EF71F070E451FF4F2081AB
:1085F00082958695877090E0032E02C0880F991FA0
:108600000A94E2F78095822380834F5F5F4FF0E00A
:108610004D375F0721F76E5F7F4F6830710521F09E
:10862000362F46E750E0DBCF80E090E00895382F0A
:10863000E82FEF71E43180F4F0E0E451FF4F208146
:1086400032953695377081E090E002C0880F991F0F
:108650003A95E2F7282B20830895382FE82FEF7101
:10866000E43188F4F0E0E451FF4F208132953695F3
:10867000377081E090E002C0880F991F3A95E2F7C9
:1086800080958223808308950F931F93CF93DF9368
:108690009C01CB01820F931F839724F062E270E06C
:1086A000621B730BD901A55FBE4FA901620F731F37
:1086B000C1E0D0E018C0FD018491E82FEF71E431F2
:1086C00078F4F0E0E451FF4F208182958695877021
:1086D0008E0102C0000F111F8A95E2F7202B208324
:1086E0004F5F5F4F1196461757072CF3DF91CF91DD
:1086F0001F910F9108950F931F93CF93DF939C01C8
:10870000CB01820F931F839724F062E270E0621B1B
:10871000730BD901A55FBE4FA901C1E0D0E01AC01B
:10872000FD018491E82FEF71E43188F4F0E0E45129
:10873000FF4F20818295869587708E0102C0000FC1
:10874000111F8A95E2F7C8018095822380834F5FCD
:108750005F4F1196461757071CF3DF91CF911F917A
:108760000F910895809164008F7E809364008FEF55
:108770008093E50087E08093E6008EE68093E70033
:1087800088EC8093E40062E270E080E090E00E9478
:108790007B0380E290E024E0959587952A95E1F7A8
:1087A000009711F481E090E09093340180933301BD
:1087B000909332018093310180E090E00895CF934F
:1087C000DF93660F771FA6E7B0E040E050E0C82FC8
:1087D000D0E0CE01042E02C0959587950A94E2F769
:1087E00080FF16C0FD018491E82FF0E0EF71F0707A
:1087F000E451FF4F208182958695877090E0062E88
:1088000002C0880F991F0A94E2F7282B208316C014
:10881000FD018491E82FF0E0EF71F070E451FF4F1B
:10882000208182958695877090E0062E02C0880F81
:10883000991F0A94E2F78095822380834F5F5F4FF0
:1088400011964730510509F0C4CFDF91CF910895BB
:10885000AF92BF92CF92DF92EF92FF920F931F934E
:10886000CF93DF937C01C62ED42EC0E0D0E000E091
:1088700010E04FE0A42EB12CF501002E02C0EE0F47
:10888000FF1F0A94E2F7EE21FF21002E02C0F695A9
:10889000E7950A94E2F7EC59FF4FE491BE018E2F61
:1088A0000E94DF032196C430D105C1F10C5F1F4F38
:1088B000C701002E02C0969587950A94E2F7892B8E
:1088C000D9F6BE01CC2089F02196DD2019F0E5E72C
:1088D000F0E002C0E4E6F0E084910E94DF03DD20D6
:1088E000C9F48091F400806803C08091F4008F7710
:1088F0008093F4000FC0DD2019F0E4E7F0E002C03F
:10890000E4E6F0E08E010F5F1F4F8491BE010E94EC
:10891000DF03E801C430D10574F30BC0CC2021F093
:108920008091F400806803C08091F4008F77809379
:10893000F40080E090E0DF91CF911F910F91FF90C4
:10894000EF90DF90CF90BF90AF900895462F28ED25
:10895000813F920714F481EF98EDFC0187E2E0314A
:10896000F80714F0EFE0F7E2DF01F7FF04C0AA27F1
:10897000BB27AE1BBF0B8A2F6AE00E94F50C282F85
:1089800030E054E0220F331F5A95E1F76F2F661F36
:108990006627661F96EF899F802D11248A0F822BF0
:1089A00090E00E9428040895462F60E00E94280469
:1089B00008950F931F93CF93DF93982F9B016830F7
:1089C00071050CF05EC08A52813520F0903209F0BA
:1089D00058C00BC0913608F09F7D903231F0892F3E
:1089E0008A52863308F04DC001C080E0E82FF0E0E5
:1089F000EE0FFF1FE358FF4F85919591A591B4911C
:108A0000EC01822F81508695A82FB0E0A451BF4F72
:108A100068E070E440E050E0890101701070FD01F1
:108A2000E40FF51FCE018F70382F962F9F7024E032
:108A3000D695C7952A95E1F784E0769567958A954E
:108A4000E1F70115110519F0292F206F06C03295A5
:108A5000307F292F2295207F2F6090818081832B6A
:108A60009223892B8083808190812823232B2923A3
:108A700020834B5F5F4F4431510589F620E030E0A1
:108A800002C02FEF3FEFC901DF91CF911F910F91EE
:108A90000895EF92FF920F931F93CF93DF937C0182
:108AA0008B01C1E0D0E005C0BE0180E20E94D90484
:108AB0002196C017D107C4F3E8010EC0F7018081E9
:108AC000882319F4BE0180E204C00894E11CF11C63
:108AD000BE010E94D9042196C830D1057CF380E004
:108AE00090E0DF91CF911F910F91FF90EF9008954B
:108AF0000F931F9300911A0110911B01F801E45E7E
:108B0000FE4F80830F5F1F4F10931B0100931A01CC
:108B1000F801E45EFE4F10828091180190911901D6
:108B200061E070E0845E9E4F0E9449051092300122
:108B3000083011051CF081E08093300180E090E066
:108B40001F910F9108951F920F920FB60F9211244B
:108B50002F933F934F935F936F937F938F939F9345
:108B6000AF93BF93EF93FF9380913001882309F473
:108B700042C080913101909132010197909332016E
:108B800080933101892BB9F5209118013091190199
:108B9000F901E45EFE4F8081882339F410921901B7
:108BA0001092180187E090E007C080910001909139
:108BB0000101009731F0019790930101809300012A
:108BC00006C02F5F3F4F3093190120931801609129
:108BD0000001709101018091180190911901845E4A
:108BE0009E4F0E94490580913301909134019093EA
:108BF000320180933101FF91EF91BF91AF919F912D
:108C00008F917F916F915F914F913F912F910F9035
:108C10000FBE0F901F901895279A2F9808952798A8
:108C20002F9A0895E4E6F0E0E80FF11DE49170E07A
:108C30008E2F0E94DF0308950F931F938C01BC01B8
:108C40008CE191E00E94D50CC8010E94DC0C8C01E3
:108C500090931B0180931A01109219011092180130
:108C600061E070E08CE191E00E94490510923001D2
:108C7000083011051CF081E08093300180E090E025
:108C80001F910F910895CF92DF92EF92FF920F9371
:108C90001F93D82EC92E5CE1E52E51E0F52E482F0A
:108CA000592FC7010E94E50C0D2D1C2D10931B019F
:108CB00000931A01109219011092180161E070E0FE
:108CC000C7010E94490510923001083011051CF0BF
:108CD00081E08093300180E090E01F910F91FF9040
:108CE000EF90DF90CF9008950F931F93182F092FC7
:108CF000682F792F8CE191E00E94EE0CE12FF02F8C
:108D0000DF010D900020E9F78D01015010400E1B8E
:108D10001F0B10931B0100931A011092190110925E
:108D2000180161E070E08CE191E00E944905109229
:108D30003001083011051CF081E08093300180E0A3
:108D400090E01F910F9108959AE0899FF0011124FE
:108D5000EE56FE4FA7E3B1E084918D93319681E00A
:108D6000A134B807C9F7089580913701909138016F
:108D700021E08D329207A1F42CE931E0A7E3B1E0C4
:108D8000F90184918D932F5F3F4FF1E0A134BF072C
:108D9000B9F780913701909138010E941C0608951F
:108DA0008553914099F422E931E0A7E3B1E0F9015C
:108DB00084918D932F5F3F4FF1E0A134BF07B9F746
:108DC00080913701909138010E941C06089580918E
:108DD0003701909138018A54914011F40E940F0B91
:108DE00080913701909138018B56914011F40E9487
:108DF000C20A80913701909138018D53914021F43E
:108E00000E94BF0A0E94EC0208951F930E94B203C1
:108E10000E94B8020E946E080E947D0B0E944D0CB9
:108E20000E94AE0C789483EE0E9417038DEE0E9490
:108E3000170322E931E0A7E3B1E0F90184918D93B2
:108E40002F5F3F4FF1E0A134BF07B9F780913701A1
:108E5000909138010E941C060E94B80C1AE0789488
:108E600080919C018823C9F110929C010E94B40654
:108E700080919601882311F00E941D0B809197012B
:108E8000882311F00E94D60A80919501882329F148
:108E900080914101843059F480919901882339F4FB
:108EA00010924101109242010E94BF0A16C08091A7
:108EB0009901882371F010929901809142018F5F8E
:108EC00080934201843049F482E392E00E941C06C0
:108ED00004C00E94C50A809341010E94A602882313
:108EE00009F48CC00E94AB02843089F1853030F4E3
:108EF000813059F0823009F07FC018C0883009F401
:108F000037C0803109F078C04AC080913B01819F11
:108F1000F0011124EE56FE4FA7E3B1E084918D934A
:108F2000319681E0A134B807C9F760C080913C0157
:108F3000819FF0011124EE56FE4FA7E3B1E084912A
:108F40008D93319681E0A134B807C9F74FC0809165
:108F50003901819FF0011124EE56FE4FA7E3B1E0E5
:108F600084918D93319681E0A134B807C9F73EC052
:108F700080913F0190914001892B89F480913A01C1
:108F8000819FF0011124EE56FE4FA7E3B1E08491DA
:108F90008D93319681E0A134B807C9F727C0E091DD
:108FA0003F01F0914001309739F180913D0190915E
:108FB0003E01099580913D0190913E01892B31F050
:108FC00080913701909138010E941C0680913A01EE
:108FD000819FF0011124EE56FE4FA7E3B1E084918A
:108FE0008D93319681E0A134B807C9F7809137019C
:108FF000909138010E941C060E94E70680E00E94C2
:1090000016092DCFFC011182818180830895DC0136
:109010009C919F5F903508F090E011968C9111978C
:10902000981731F08C91FD01E80FF11D62839C933C
:109030000895DC0111968C911197FD01E80FF11D47
:1090400092818F5F803508F080E011968C93892F94
:109050000895109243018091430180934401089543
:10906000FC019081818120E0981321E0822F0895F6
:109070008A3010F0895C0895805D0895FB0190E3CB
:1090800090838F708A3010F0895C01C0805D81838D
:10909000089520E43BE44CE450E00BC02115310579
:1090A0004105510511F49FEF17C021503040404059
:1090B00050409091430180914401981779F3809139
:1090C0004401E82FF0E0ED5BFE4F92818F5F803529
:1090D00008F080E080934401892F0895E4E6F0E0F1
:1090E00080818D7F80831092430180914301809322
:1090F00044018CE090E09093C5008093C40086E02A
:109100008093C20088E98093C10008951092C10045
:10911000E4E6F0E08081826080830895982F80915A
:10912000C00085FFFCCF9093C60008951F920F9258
:109130000FB60F9211242F938F939F93EF93FF936A
:109140002091C600909143019F5F903508F090E018
:1091500080914401981741F0E0914301F0E0ED5B0C
:10916000FE4F228390934301FF91EF919F918F9146
:109170002F910F900FBE0F901F901895982F8091F0
:10918000C00085FFFCCF81E08093C6008091C000C5
:1091900085FFFCCF6093C6008091C00085FFFCCFA7
:1091A0009093C600FA0190E009C020818091C00030
:1091B00085FFFCCF2093C6009F5F31969617A9F7D5
:1091C0008091C00085FFFCCF84E08093C6000895A5
:1091D000DF93CF93CDB7DEB764970FB6F894DEBFB9
:1091E0000FBECDBF982FDE011196E2E0F1E088E0DE
:1091F00001900D928150E1F7FE0139968CE0DF017C
:109200001D928A95E9F7BE016C5F7F4F892F0E94FE
:10921000790ACE0101960E94740664960FB6F894FE
:10922000DEBF0FBECDBFCF91DF910895DF93CF9307
:10923000CDB7DEB72D970FB6F894DEBF0FBECDBF0A
:10924000882399F49091430180914401981769F41F
:1092500047C1211531054105510511F49FEF1CC08F
:10926000215030404040504004C020E43BE44CE4F6
:1092700050E09091430180914401981751F38091FF
:109280004401E82FF0E0ED5BFE4F92818F5F803567
:1092900008F080E08093440199838981813011F046
:1092A00081E0EDC00E940C0620E43BE44CE450E079
:1092B0000BC0211531054105510511F49FEF17C071
:1092C00021503040404050409091430180914401F2
:1092D000981779F380914401E82FF0E0ED5BFE4FA1
:1092E00092818F5F803508F080E0809344019983FC
:1092F00089818F3F11F482E0C2C0898187FF2CC031
:1093000020E43BE44CE450E00BC02115310541055D
:10931000510511F49FEF17C021503040404050409C
:109320009091430180914401981779F38091440111
:10933000E82FF0E0ED5BFE4F92818F5F803508F003
:1093400080E08093440199838981843009F4C6C008
:1093500083E00E94E808C2C089818A838A818B30B9
:1093600008F0BEC020E43BE44CE450E00BC0211503
:1093700031054105510511F49FEF17C021503040D0
:10938000404050409091430180914401981779F3F7
:1093900080914401E82FF0E0ED5BFE4F92818F5FFA
:1093A000803508F080E080934401998389818F3F64
:1093B00011F485E064C089818B8360E070E0DE0198
:1093C00014962BC0211531054105510511F49FEF6D
:1093D00017C021503040404050409091430180914F
:1093E0004401981779F380914401E82FF0E0ED5B98
:1093F000FE4F92818F5F803508F080E080934401BA
:10940000998389818F3F11F4862F39C08981FD01AD
:10941000E60FF71F80836F5F7F4F8A8190E06817A8
:10942000790728F020E43BE44CE450E010C020E44D
:109430003BE44CE450E0D1CF211531054105510505
:1094400011F49FEF17C021503040404050409091A0
:10945000430180914401981779F380914401E82FEA
:10946000F0E0ED5BFE4F92818F5F803508F080E089
:109470008093440199838981843021F087E00E94A0
:10948000E8082EC08B81813CD1F0823C09F1803C00
:1094900029F58C8180939B01813011F463E00BC02E
:1094A000823011F462E007C0833011F461E003C040
:1094B000843019F460E00E9412061092990181E54F
:1094C0000E9417030E94250C81E50E942D0306C00F
:1094D000CE0104960E9474060E94250C0E940F067D
:1094E0002D960FB6F894DEBF0FBECDBFCF91DF91A2
:1094F0000895282FFB016AE00E94F50C905D91838E
:10950000822F0E94F50C805D808308959C01FB01F1
:1095100097FD02C040E004C0309521953F4F41E0E7
:109520001082319780919A01DF011197882311F4FD
:1095300083E401C086E4808380E28C93FD0131974F
:109540002115310519F480E3808317C0C9016AE051
:1095500070E00E94010D805D80833197C9016AE04F
:1095600070E00E94010D9B016115710579F744239C
:1095700019F08DE2808331973196CF0108951092D2
:109580009501089510929701089581E080939901C3
:10959000809198018F5F8093980148E951E061E0E4
:1095A00081E80E94BE08809198010895DF93CF93CF
:1095B000CDB7DEB72A970FB6F894DEBF0FBECDBF8A
:1095C0000E940C0680919A010E945F0CBE01655FAB
:1095D0007F4F0E94860ADC010D900020E9F7119769
:1095E000A81BB90BAC016A2F80E80E94BE080E943C
:1095F0000F062A960FB6F894DEBF0FBECDBFCF91EF
:10960000DF910895FC018081882319F01092970161
:1096100003C081E0809397010E94D60A08951092BA
:10962000960180E50E942D0380ED0E942D0382EEBD
:109630000E942D030E94EC020895CF93DF93809146
:109640009A010E945F0CEC0180919A01882329F411
:1096500080E50E942D0380ED04C080ED0E942D0363
:1096600080E50E94170305B607FE04C082EE0E9443
:109670002D0303C082EE0E94170361E0CE010E9419
:10968000A604DF91CF910895FC018081882319F011
:1096900010929A0103C081E080939A0181E0809347
:1096A00096010E941D0B08951F93FC011FB7F894AB
:1096B0008081882371F085B7806885BF85B7806811
:1096C00085BF0E944D0CF999FECF12BC11BC8FEFE3
:1096D0000BC085B78F7785BF85B78F7785BFF99921
:1096E000FECF12BC11BC81E080BD0FB6F894FA9A8F
:1096F000F99A0FBE1FBF1F910895DF93CF930F926A
:10970000CDB7DEB7F999FECF12BC11BCF89A80B57F
:109710009E012F5F3F4F8F3F19F481E0898301C085
:109720001982C9010E94540B0F90CF91DF910895C7
:1097300081E0809395011092980110929B0160E066
:1097400081E10E94120661E081E10E94120662E05E
:1097500081E10E94120663E081E10E9412060E94EC
:10976000C50A10928500109284000895DF93CF936C
:1097700000D0CDB7DEB79A8389830E940F0680910F
:1097800064008C60809364000E94C8020E94B5024D
:109790000E94EA0B0E94B2038FE392E00E941C0633
:1097A00083EE0E9417030E94B8020E940F0C0E94D1
:1097B0006F028823E1F70E94A602882311F00E941D
:1097C000AB02CE0101960E941C060F900F90CF9124
:1097D000DF91089588E10FB6F894809360001092AD
:1097E00060000FBE83B7817F846083BFEC9AEBE695
:1097F000F0E080818460808383B7816083BF889537
:1098000083B78E7F83BFEC9808951F920F920FB697
:109810000F9211240F900FBE0F901F90189502C049
:109820000E94490890914301809144019817C1F723
:1098300088E70E948E089091430180914401981717
:10984000B9F381E00E9416090895DF93CF930F9238
:10985000CDB7DEB76F9A779A259A90E01D9A198254
:1098600003C089818F5F898389818F3FD1F79F5F93
:109870009436A1F790E01D9A198203C089818F5F09
:1098800089838981803AD0F39F5F9436A1F72D9820
:1098900077980F90CF91DF910895EEE7F0E0808107
:1098A00080618083869A8E9884988C9881E08093DA
:1098B000360180E090E008951092360108951F93DC
:1098C000CF93DF93182F80913601882309F43FC08E
:1098D0008E9A27E040E460E084E00E941C020E942F
:1098E000400280E00E945302EC018FEFCF3FD80787
:1098F000C1F30E9431020E94B8028E981123B1F484
:1099000047E452E020E030E0FA01859194918C1711
:109910009D074CF02F5F3F4F4E5F5F4F2C3431055A
:1099200099F72FEF3FEF2F50304013C04FED52E02B
:1099300020E030E0FA01859194918C179D074CF05E
:109940002F5F3F4F4E5F5F4F2D38310599F72FEF57
:109950003FEFC901DF91CF911F9108958DE0809372
:10996000810084E89EE190938900809388000895A7
:10997000109285001092840082E080936F00089519
:10998000EFE6F0E080818D7F808308951F920F9233
:109990000FB60F9211248F9381E080939C018F91D9
:1099A0000F900FBE0F901F901895FB01DC010590E2
:1099B0000D920020E1F70895FC0105900020E9F7E1
:1099C000809590958E0F9F1F0895FB01DC0102C0CA
:1099D00001900D9241505040D8F70895FB01DC01F1
:1099E00001900D920020E1F70895991B79E004C0E1
:1099F000991F961708F0961B881F7A95C9F78095CE
:109A0000089597FB092E07260AD077FD04D00CD0C5
:109A100006D000201AF4709561957F4F0895F6F7EF
:109A2000909581959F4F0895AA1BBB1B51E107C0DC
:109A3000AA1FBB1FA617B70710F0A61BB70B881FDE
:109A4000991F5A95A9F780959095BC01CD0108956D
:109A5000F894FFCF0100544F202020202000000068
:109A600000000000000000000000E299FF1C000060
:109A700000020000000000040000000000380400A4
:109A800000A600000000000000000000001C000014
:109A900000020052020000040000000000DE04008A
:109AA00000B200000000000000000000001C0000E8
:109AB000000200B604000004000000000090050051
:109AC00000B807000000000000000000001C0000BB
:109AD0000002000D140000040000000000480D000A
:109AE00000BC02000000000000000000001C00009C
:109AF00000FFFFFFFFFFFFFFFFFFFFFFFFFFFFFF75
:109B0000FFFFFFFFFFFFFFFFFFFFFFFFFFFFFFFF65
:109B1000FFFFFFFFFFFFFFFFFFFFFFFFFFFFFFFF55
:109B2000FFFFFFFFFFFFFFFFFFFFFFFFFFFFFFFF45
:109B3000FFFFFFFFFFFFFFFFFFFFFFFFFFFFFFFF35
:00000001FF
